:100000000C942C030C9454030C9454030C9435134B
:100010000C9435130C9435130C9454030C94540322
:100020000C9454030C9454030C9454030C945403F4
:100030000C9454030C9454030C9454030C945403E4
:100040000C94EB120C9454030C94EA110C94C4110C
:100050000C9454030C9454030C9454030C945403C4
:100060000C9454030C94540305A84CCDB2D44EB94F
:100070003836A9020C50B9918688083CA6AAAA2A4B
:10008000BE000000803F04E010021C071237322936
:100090002D29252B3900010310E110031D07062E21
:1000A0002C292D2E2E373F0000021013800A2980A4
:1000B00064022A040000007F2B040000009F0F014F
:1000C00080961180FFB103012C2DB203012C2DB3BA
:1000D00006012C2D012C2DB40107C003A20284C1FE
:1000E00001C5C2020A00C3028A2AC4028AEEC501FF
:1000F0000E20003601C83A010500000000003E5BFA
:100100004F5B3E3E6B4F6B3E1C3E7C3E1C183C7E64
:100110003C181C577D571C1C5E7F5E1C00183C1849
:1001200000FFE7C3E7FF0018241800FFE7DBE7FF45
:1001300030483A060E2629792926407F05050740D2
:100140007F05253F5A3CE73C5A7F3E1C1C08081C93
:100150001C3E7F14227F22145F5F005F5F06097FD1
:10016000017F006689956A606060606094A2FFA26A
:100170009408047E040810207E201008082A1C0819
:10018000081C2A08081E101010100C1E0C1E0C3023
:10019000383E3830060E3E0E06000000000000001B
:1001A0005F00000007000700147F147F14242A7FDB
:1001B0002A122313086462364956205000080703A8
:1001C00000001C2241000041221C002A1C7F1C2A26
:1001D00008083E0808008070300008080808080079
:1001E0000060600020100804023E5149453E004274
:1001F0007F400072494949462141494D3318141244
:100200007F1027454545393C4A494931412111096B
:10021000073649494936464949291E00001400005D
:100220000040340000000814224114141414140077
:100230004122140802015909063E415D594E7C12C3
:1002400011127C7F494949363E414141227F41415B
:10025000413E7F494949417F090909013E414151D8
:10026000737F0808087F00417F41002040413F0123
:100270007F081422417F404040407F021C027F7F64
:100280000408107F3E4141413E7F090909063E4175
:1002900051215E7F09192946264949493203017FC8
:1002A00001033F4040403F1F2040201F3F40384057
:1002B0003F631408146303047804036159494D43F0
:1002C000007F4141410204081020004141417F0468
:1002D000020102044040404040000307080020544F
:1002E0005478407F284444383844444428384444AF
:1002F000287F385454541800087E090218A4A49C7E
:10030000787F0804047800447D40002040403D0090
:100310007F1028440000417F40007C047804787CF2
:10032000080404783844444438FC18242418182459
:100330002418FC7C08040408485454542404043F42
:1003400044243C4040207C1C2040201C3C40304049
:100350003C44281028444C9090907C4464544C4475
:100360000008364100000077000000413608000216
:10037000010204023C2623263C1EA1A161123A4040
:1003800040207A38545455592155557941225454B6
:100390007842215554784020545579400C1E5272B1
:1003A000123955555559395454545939555454588E
:1003B0000000457C410002457D420001457C407DB6
:1003C0001211127DF0282528F07C54554500205448
:1003D000547C547C0A097F4932494949323A4444A1
:1003E000443A324A4848303A4141217A3A42402020
:1003F00078009DA0A07D3D4242423D3D4040403DB1
:100400003C24FF2424487E4943662B2FFC2F2BFFDE
:100410000929F620C0887E09032054547941000040
:10042000447D413048484A32384040227A007A0AB6
:100430000A727D0D19317D2629292F28262929297F
:100440002630484D402038080808080808080838B1
:100450002F10C8ACBA2F102834FA00007B00000817
:10046000142A142222142A14085500550055AA559E
:10047000AA55AAFF55FF55FF000000FF00101010FD
:10048000FF00141414FF001010FF00FF1010F010F4
:10049000F0141414FC001414F700FF0000FF00FF18
:1004A0001414F404FC141417101F10101F101F1440
:1004B00014141F00101010F0000000001F10101086
:1004C000101F10101010F010000000FF101010107E
:1004D0001010101010FF10000000FF140000FF00AB
:1004E000FF00001F10170000FC04F414141710176D
:1004F0001414F404F40000FF00F71414141414147A
:1005000014F700F7141414171410101F101F1414EC
:1005100014F4141010F010F000001F101F00000061
:100520001F14000000FC140000F010F01010FF1069
:10053000FF141414FF141010101F00000000F0101E
:10054000FFFFFFFFFFF0F0F0F0F0FFFFFF00000003
:100550000000FFFF0F0F0F0F0F3844443844FC4AD0
:100560004A4A347E02020606027E027E0263554932
:1005700041633844443C04407E201E2006027E0233
:100580000299A5E7A5991C2A492A1C4C7201724CB4
:10059000304A4D4D303048784830BC625A463D3E76
:1005A000494949007E0101017E2A2A2A2A2A444417
:1005B0005F444440514A444040444A51400000FF97
:1005C0000103E080FF000008086B6B083612362438
:1005D00036060F090F060000181800000010100062
:1005E0003040FF0101001F01011E00191D171200FC
:1005F0003C3C3C3C000000000000000000240027C0
:10060000002A0000000008000201000003040700A7
:100610000000000000000000000000250028002B62
:100620000000000000230026002900040404040444
:10063000040404020202020202030303030303018F
:100640000204081020408001020408102001020466
:1006500008102000742F5B2E11241FBECFEFD8E0AE
:10066000DEBFCDBF13E0A0E0B1E0EAE1F8E602C0F2
:1006700005900D92AE33B107D9F724E0AEE3B3E0B5
:1006800001C01D92AF39B207E1F713E0CBE2D3E02E
:1006900004C02197FE010E94F533CA32D107C9F781
:1006A0000E94691A0C9400340C9400000895FC0117
:1006B0006370658B8481958126813781613039F043
:1006C000633029F0918780873387228708953187A7
:1006D00020879387828708952F923F924F925F924F
:1006E0006F927F928F929F92AF92BF92CF92DF9242
:1006F000EF92FF920F931F93CF93DF93CDB7DEB7A7
:100700006C970FB6F894DEBF0FBECDBF9C8F8B8F5A
:100710001B012A0118870F83FE82ED82CA82DC0149
:1007200058964D915C9159974115510509F0B2C009
:1007300018968D919C911997681779070CF096C1BE
:100740001A968D919C911B97481659060CF08EC1F4
:10075000AC2CB12CCB01B6E0CB9E800D911D1124A9
:10076000181619060CF082C1C50133E0880F991FD5
:100770003A95E1F7840D951D181619060CF076C10F
:10078000AB8DBC8D57968C91811103C0203B08F036
:100790002F5FAB8DBC8DED91FC9111970680F78199
:1007A000E02DCD012A8F09952A8DB5E02B9F900170
:1007B0001124610141011B82F901E219F309FA8751
:1007C000E9879201285F3F4F3C872B873B8135307B
:1007D00049F0E985FA85E80DF91DE750FF4F44918E
:1007E000498301C0198232011201598150FF13C09F
:1007F000AB8DBC8DED91FC91BA81B13031F40084A8
:10080000F185E02D2F81388519C00284F385E02D14
:10081000EF80F8841EC0ED81FE812F813885E217BC
:10082000F307F1F0AB8DBC8DED91FC91BA81B13045
:1008300059F40084F185E02D2D813E81A301B4019E
:100840008B8D9C8D09950CC00284F385E02DED8085
:10085000FE8085019501A101B6018B8D9C8D0995C6
:10086000E981E695E983FFEF6F1A7F0A2A0C3B1CAA
:100870002B853C856216730609F0B7CF3B813F5F3D
:100880003B834FEF841A940ACA0CDB1C363009F004
:100890009DCFCAC0FA0134969491329765917491B4
:1008A000291BCB01B7E02B9F800D911D1124FA016C
:1008B000259134913A8B298BFC0165907490FC0151
:1008C000329634913D83319644914B873296C49051
:1008D000319614915A81523058F08C2C0C2C000C0B
:1008E0009908812F012E000C990B9C838B8304C0E7
:1008F0001C821B82812C912CAB8DBC8DED91FC91C7
:1009000011970680F781E02DCD010995BA81AB2EB4
:10091000B12C8A9CC0018B9C900D9A9C900D112447
:10092000FC01E20DF31DF88BEF871982912C812CCD
:10093000EC2DCC0CFF0B91012E0F3F1F3A8729871E
:1009400061013D81C30ED11CA6014E0F5F1F5F8B5D
:100950004E8BC201810F911D17FD9A95998F888F3B
:100960005B85851608F060C0882D90E04B815C8126
:10097000480F591F4A9D90014B9D300D5A9D300DD7
:100980001124D901A40DB51DBE87AD87C984DA84B1
:100990002F843888B981E985BE1BBB8B288D398DA2
:1009A000280F391F3D8B2C8B8B898C0D2E893F890D
:1009B000C216D30699F1877041F4C3010196E98903
:1009C000FA89E60DF71D94903C0197FE20C0AB8D8F
:1009D000BC8DED91FC91BA81B13061F40084F18558
:1009E000E02D2F8138854C895D89B6018B8D9C8DDA
:1009F00009950DC00284F385E02DEF80F884850110
:100A000095014D855E85B1018B8D9C8D0995990C65
:100A1000EFEFCE1ADE0A2A0C3B1CC6CF39814D817E
:100A2000340F398383949CCFAB8DBC8DED91FC91B9
:100A300011970288F389E02DCD016C960FB6F894DA
:100A4000DEBF0FBECDBFDF91CF911F910F91FF9001
:100A5000EF90DF90CF90BF90AF909F908F907F905E
:100A60006F905F904F903F902F9009946C960FB6C7
:100A7000F894DEBF0FBECDBFDF91CF911F910F91D4
:100A8000FF90EF90DF90CF90BF90AF909F908F90AE
:100A90007F906F905F904F903F902F900895AF920E
:100AA000BF92CF92EF92FF920F931F93CF93DF935A
:100AB000EC01262F888D998D009709F042C06A308D
:100AC00069F42C898E859F8538E0239F800D911DC8
:100AD00011249F878E871D861C86ACC06D3009F45B
:100AE000A9C08E898823C1F03C898C859D8546E00C
:100AF000349F800D911D11244885598584179507D1
:100B00005CF01D861C868E859F85E8E03E9F800DEB
:100B1000911D11249F878E87EA88FB88088919898F
:100B20004E855F856C857D85CC88CE010E946C03E7
:100B30002C898C859D85F6E02F9F800D911D1124B9
:100B400041C06A3079F41D861C862C89FC013696DA
:100B5000E4918E859F852E9F800D911D11249F8786
:100B60008E8768C06D3009F465C0AC014C5F5F4F83
:100B7000FA013491631708F45DC03196E491E617E9
:100B800008F458C0FA014491362F341BFC01329608
:100B9000A590B490F7E03F9FA00CB11C1124F50183
:100BA000329634913196E491332311F0E1110DC066
:100BB000F5013496E4912C898C859D85E29F800D0A
:100BC000911D11249D878C8735C0F5013596449180
:100BD0005E89552311F16C89E32FF0E0E40FF11DDC
:100BE00047FDFA956E9FD0016F9FB00D11244C8583
:100BF0005D854A0F5B1FE885F9854E175F076CF02E
:100C00001D861C86FC013696E4918E859F856E9F1D
:100C1000800D911D11249F878E87EA88FB880889A3
:100C200019894E855F856C857D85CC88CE010E94B3
:100C30006C03BECF81E090E0DF91CF911F910F91C7
:100C4000FF90EF90CF90BF90AF9008956F927F92FA
:100C50008F929F92AF92BF92CF92DF92EF92FF92CC
:100C60000F931F93CF93DF93EC014B015A0169015E
:100C70003801E881F9810680F781E02D0995E88146
:100C8000F9810684F785E02D87019601A501B4015D
:100C9000CE010995E881F981A501460D571D415006
:100CA00051090684F785E02D9601B401CE0109951E
:100CB000E881F9810484F585E02D9301A501B40153
:100CC000CE010995E881F981C80CD91CB6016150A3
:100CD00071090484F585E02D9301A501CE010995E4
:100CE000E881F9810288F389E02DCE01DF91CF916F
:100CF0001F910F91FF90EF90DF90CF90BF90AF903A
:100D00009F908F907F906F900994CF92DF92EF9297
:100D1000FF920F931F93CF93DF9300D000D000D0AA
:100D2000CDB7DEB76C01DC01ED91FC916217730762
:100D300089F4041715072CF4942F852FA801092F87
:100D4000182F041B150B98012F5F3F4F008CF18D5E
:100D5000E02D12C04017510709F5261737072CF46C
:100D6000962F872FB901292F382F261B370B2F5F7E
:100D70003F4F028CF38DE02D8701C6010995269621
:100D80000FB6F894DEBF0FBECDBFDF91CF911F919C
:100D90000F91FF90EF90DF90CF9008950680F7813C
:100DA000E02D2D833E834B835C8369837A83099591
:100DB000D601ED91FC910088F189E02D2D813E81D5
:100DC0004B815C8169817A81C6010995D601ED91DB
:100DD000FC910288F389E02DC60126960FB6F8949F
:100DE000DEBF0FBECDBFDF91CF911F910F91FF905E
:100DF000EF90DF90CF900994EF92FF920F931F93A3
:100E0000DC01ED91FC9111971A960D911C911B97A5
:100E100018962D913C911997048CF58DE02D7B014E
:100E200040E050E060E070E009951F910F91FF9065
:100E3000EF9008954F925F926F927F928F929F9260
:100E4000AF92BF92CF92DF92EF92FF920F931F93D8
:100E5000CF93DF9300D0CDB7DEB76C015A013901D3
:100E60004801DC01ED91FC910680F781E02D69835A
:100E70007A8309956981462E7A81572E640C751CF8
:100E8000D601ED91FC91461457046CF40484F58569
:100E9000E02D87019401A501B201C6010995BFEFBC
:100EA0004B1A5B0AEDCF0288F389E02DC6010F9043
:100EB0000F90DF91CF911F910F91FF90EF90DF90F6
:100EC000CF90BF90AF909F908F907F906F905F90EA
:100ED0004F900994AF92BF92CF92DF92EF92FF9220
:100EE0000F931F93CF93DF9300D000D0CDB7DEB721
:100EF0005C016901DC01ED91FC910680F781E02D38
:100F00004B835C8369837A830995D501ED91FC91CC
:100F100069817A819B012C0D3D1D2150310900888A
:100F2000F189E02D78014B815C818A01C501099529
:100F3000D501ED91FC910288F389E02DC5010F9058
:100F40000F900F900F90DF91CF911F910F91FF9015
:100F5000EF90DF90CF90BF90AF900994AF92BF9287
:100F6000CF92DF92EF92FF920F931F93CF93DF9375
:100F700000D000D0CDB7DEB75C016901DC01ED9196
:100F8000FC910680F781E02D4B835C8369837A8333
:100F90000995D501ED91FC914B815C81C40ED51E64
:100FA000B1E0CB1AD1080088F189E02D78018601E3
:100FB00069817A819B01C5010995D501ED91FC916B
:100FC0000288F389E02DC5010F900F900F900F90CC
:100FD000DF91CF911F910F91FF90EF90DF90CF9015
:100FE000BF90AF9009940895EF92FF920F931F93D3
:100FF000DC01ED91FC91048CF58DE02D09951F919C
:101000000F91FF90EF9008950F931F93DC01ED91E6
:10101000FC91028CF38DE02D09951F910F9108959D
:101020000F931F93DC01ED91FC91008CF18DE02D6D
:1010300009951F910F910895DC01ED91FC910480B9
:10104000F581E02D099408952F923F924F925F927F
:101050006F927F928F929F92AF92BF92CF92DF92C8
:10106000EF92FF920F931F93CF93DF9300D01F92C5
:10107000CDB7DEB74C017B836A836A015901170142
:101080009801241B350B37FF03C031952195310999
:10109000C5014A815B81841B950B97FF03C0919525
:1010A0008195910951E059838217930714F01982B1
:1010B0000BC09A2D8B2D5801092F182F9A818B81E7
:1010C000DB82CA82C92ED82E8A819B81A816B906D6
:1010D0005CF49C2D8D2D6801092F182F9A818B812E
:1010E000BB82AA82A92EB82E2501AA81BB814A1AE9
:1010F0005B0A38016C187D0877FE03C07194619417
:101100007108720157FE03C0BFEFEB1AFB0AF5949A
:10111000E794C016D1061CF00FEF1FEF1FC001E0CF
:1011200010E01CC0D401ED91FC91B9810084F185DF
:10113000E02D9101BB23C1F04A815B81B601C4015E
:101140000995E618F708F7FE04C0C00ED11EE40C9E
:10115000F51CEA81FB813196FB83EA834A815B813E
:10116000A416B506FCF604C0A6016A817B81E7CF10
:101170000F900F900F90DF91CF911F910F91FF90E3
:10118000EF90DF90CF90BF90AF909F908F907F9027
:101190006F905F904F903F902F900895FC01838D4A
:1011A000882339F06EBD00000DB407FEFDCF8EB56B
:1011B000089528E030E090E8A48DB58D81A5492FF1
:1011C000462319F04C91842B03C04C9180958423C5
:1011D0008C93A68DB78D4C9182A5842B8C93A68D74
:1011E000B78D4C9182A5809584238C939695215040
:1011F000310911F7089508958CBD9DBD08950F9391
:101200001F93CF93DF931F92CDB7DEB78C018091F0
:101210004B0490914C0469830E94FC08D80192967B
:10122000ED91FC91939790819C968C919C97892B42
:1012300080839096ED91FC91919790819B968C91F3
:101240008095892380836981C8010E94CE08D801D6
:101250009096ED91FC91919790819B968C91892B22
:1012600080830F90DF91CF911F910F9108950F937D
:101270001F93CF93DF931F92CDB7DEB78C01809180
:101280004B0490914C0469830E94FC08D80192960B
:10129000ED91FC91939790819C968C919C97809571
:1012A000892380839096ED91FC91919790819B96F4
:1012B0008C918095892380836981C8010E94CE0822
:1012C000D8019096ED91FC91919790819B968C918D
:1012D000892B80830F90DF91CF911F910F910895FB
:1012E000EF92FF920F931F93CF93DF9300D0CDB770
:1012F000DEB77C01162F6AE229834A830E943709F0
:1013000060E0C7010E94FF08F70185A5612F680F03
:10131000C7010E94FF0860E0C7010E94FF08F701B3
:1013200085A52981622F680FC7010E94FF086BE223
:10133000C7010E94370960E0C7010E94FF08F7015A
:1013400086A54A81642F680FC7010E94FF0860E0EC
:10135000C7010E94FF08F70186A5602F680FC7012B
:101360000E94FF086CE2C7010F900F90DF91CF91B0
:101370001F910F91FF90EF900C943709DF92EF923D
:10138000FF920F931F93CF93DF93EC017901D02E3F
:101390008885998568177907ECF52A853B8542177A
:1013A0005307C4F59B012E0D3F1D821793071CF4B4
:1013B0007C01E61AF70A2FEF260F2E0D042FCE011F
:1013C0000E94700980914B0490914C040E94FC088B
:1013D000EAA1FBA190818CA5892B8083E8A1F9A1CA
:1013E00090818BA5809589238083E114F10461F0BD
:1013F000612FCE010E94CE086D2DCE010E94CE0835
:1014000081E0E81AF108F1CFE8A1F9A190818BA55C
:10141000892B8083DF91CF911F910F91FF90EF90E7
:10142000DF900895DF92EF92FF920F931F93CF9377
:10143000DF93EC017901D02E8885998568177907AB
:10144000ECF58A859B8548175907C4F59A012E0D3E
:101450003F1D821793071CF47C01E41AF50A0FEF75
:10146000040F0E0D262FCE010E94700980914B04AF
:1014700090914C040E94FC08EAA1FBA190818CA5EC
:10148000892B8083E8A1F9A190818BA58095892380
:101490008083E114F10461F0612FCE010E94CE0837
:1014A0006D2DCE010E94CE0881E0E81AF108F1CF3F
:1014B000E8A1F9A190818BA5892B8083DF91CF9141
:1014C0001F910F91FF90EF90DF900895EF92FF92A0
:1014D0000F931F93CF93DF931F92CDB7DEB77C019D
:1014E000CB01122F77FD49C0D70118966D917C91E1
:1014F0001997861797070CF040C057FD3EC01A9603
:101500006D917C911B9746175707BCF501E0040FBE
:1015100021E0280F682FC70139830E94700980914C
:101520004B0490914C040E94FC08D7019296ED91D7
:10153000FC91939790819C968C919C97892B8083AA
:101540009096ED91FC91919790819B968C918095CE
:10155000892380833981632FC7010E94CE08612FC0
:10156000C7010E94CE08D7019096ED91FC9191970A
:1015700090819B968C91892B80830F90DF91CF91E6
:101580001F910F91FF90EF90089580E894E00E94E2
:10159000AF130E94061867E672E08EEA93E00E949D
:1015A000AE116CEF80E894E00E94D00F62E070E032
:1015B00080E090E00C94B11260E070E081E594E08E
:1015C0000C945D10CF93DF9310927F0410927E04F1
:1015D00061E0809176040E94751261E0809175044B
:1015E0000E9475122091750430E0F901E55DF94F14
:1015F000E491F0E0EE0FFF1FE95EF94F85919491C1
:1016000090937204809371044091760450E0FA0143
:10161000E55DF94F8491E82FF0E0EE0FFF1FE95EE2
:10162000F94F859194919093740480937304F90118
:10163000E15CF94FE491E0937C04FA01E15CF94F3D
:10164000E491E0937D0480916C04882309F43AC00E
:10165000CFB7F89480915C03811127C0E5E3F6E0F1
:101660008491E9E4F6E09491E82FF0E0EE0FFF1F9B
:10167000E750FA4FA591B491EC91E92321F461E090
:101680008AE00E94451261E08AE00E9475128CB5E2
:1016900080618CBD8CB580648CBD61E08DE00E9462
:1016A000751261E08BE00E94751280915C038F5F80
:1016B00080935C03CFBF80E580934B0481E08093EF
:1016C0004C0448C061E0809179040E94751261E089
:1016D000809178040E9475128091790490E0FC0159
:1016E000E55DF94FE491F0E0EE0FFF1FE95EF94F81
:1016F000A591B491B0937004A0936F0420917804E5
:1017000030E0F901E55DF94FE491F0E0EE0FFF1FE5
:10171000E95EF94F4591549150936E0440936D04E6
:10172000FC01E15CF94F849180937B04F901E15C59
:10173000F94FE491E0937A04EC9180958E238C9399
:10174000E0916D04F0916E04908180917A0480950F
:1017500089238083E0917104F091720490818091DB
:101760007C0480958923808380917704882321F1EC
:1017700061E00E94751261E0809177040E94451239
:1017800064EF71E080E090E00E94B11260E080912F
:1017900077040E94451264EF71E080E090E00E94BF
:1017A000B11261E0809177040E94451264EF71E00C
:1017B00080E090E00E94B1128EEB90E00E942F1921
:1017C00081EB90E00E942F1986E890E00E942F198B
:1017D00066E381E594E00E94370960EC81E594E0DE
:1017E0000E94FF0882E080936B048091500490E097
:1017F0000E94D51860E070E081E594E00E945D10E1
:1018000086E00E941C1280934303813039F490914A
:101810004D04933008F483E080934D0480914D048F
:10182000833018F481E080934D0460914D0481E58C
:1018300094E00E94841082E080936504C3E1D0E0CC
:10184000D0935E04C0935D048CE190E090936004BB
:1018500080935F0480EA9DEF909364048093630417
:10186000909362048093610463E772E081E594E001
:101870000E94C211D0935E04C0935D048BE190E09E
:101880009093600480935F0480EE9FEF90936404D4
:1018900080936304909362048093610463E772E031
:1018A00081E594E00E94C21184E190E090935E048F
:1018B00080935D048DE190E09093600480935F04D9
:1018C00080E098EF909364048093630490936204A3
:1018D0008093610463E772E081E594E00E94C211A5
:1018E0006AE070E080E090E00E94B11280E894E04D
:1018F0000E94AF130E9406186AED71E08EEA93E031
:101900000E94AE116EE772E08EEA93E00E94AE1183
:1019100069E872E08EEA93E00E94AE116FEF80E812
:1019200094E00E94D00F64E170E080E090E00E94BB
:10193000B11280E894E00E942410892BC1F180E864
:1019400094E00E943C10EC0166ED71E08EEA93E0B9
:101950000E94C211BE018EEA93E00E949F186AE0C5
:1019600070E080E090E00E94B11220913F0330913E
:1019700040032115310529F4D0934203C09341035C
:101980000FC02130310529F4D0936003C0935F0369
:1019900007C02430310521F4D0935E03C0935D036A
:1019A0002F5F3F4F3093400320933F03C2CF1092ED
:1019B000400310923F0368EC70E080E090E00E94EA
:1019C000B11280EE9FEF9093640480936304909330
:1019D00062048093610481E0809365048AE090E072
:1019E00090935E0480935D048CE390E09093600498
:1019F00080935F0465E972E081E594E00E94C21182
:101A000080915F0390916003892B31F46DE972E05E
:101A100081E594E00E94C21180915F039091600380
:101A2000019731F464EA72E081E594E00E94C2110A
:101A300080915F0390916003029731F468EA72E04D
:101A400081E594E00E94C21180915F039091600350
:101A5000039731F46CEA72E081E594E00E94C211D0
:101A600080915F0390916003049731F460EB72E022
:101A700081E594E00E94C2118AE090E090935E04B8
:101A800080935D0488E490E09093600480935F0409
:101A900065EB72E081E594E00E94C2118091410300
:101AA00090914203019731F46DEB72E081E594E08F
:101AB0000E94C2118091410390914203029731F438
:101AC00061EC72E081E594E00E94C21180914103D3
:101AD00090914203039731F467EC72E081E594E062
:101AE0000E94C2118091410390914203049731F406
:101AF0006DEC72E081E594E00E94C2118091410397
:101B000090914203059731F465ED72E081E594E030
:101B10000E94C2118091410390914203069731F4D3
:101B20006BED72E081E594E00E94C2118091410367
:101B300090914203449731F468EA72E081E594E0C1
:101B40000E94C2118091410390914203459731F464
:101B500064EE72E081E594E00E94C211809141033D
:101B600090914203469731F46CEE72E081E594E087
:101B70000E94C2118AE090E090935E0480935D041D
:101B800084E590E09093600480935F0465EF72E0D9
:101B900081E594E00E94C21160915D0370915E0343
:101BA00081E594E00E949F1880915D0390915E030F
:101BB00005972CF088E28093060180933E0380EA2B
:101BC0009DEF9093640480936304909362048093E8
:101BD000610481E0809365048EE190E090935E045F
:101BE00080935D048CE690E09093600480935F04A2
:101BF00068E073E081E594E00E94C21182E891E818
:101C000090936404809363049093620480936104CE
:101C100010925E0410925D0488E790E09093600457
:101C200080935F046AE173E081E594E00E94C21151
:101C30004091500450E060E070E02AE081E594E0DB
:101C40000E94651162E273E081E594E00E94C21196
:101C500040914F0450E060E070E02AE081E594E0BC
:101C60000E9465116DE273E081E594E00E94C2116B
:101C700040914E0450E060E070E02AE081E594E09D
:101C80000E94651160E373E081E594E00E94C21157
:101C90006CEA7DE080E090E00E94B112DF91CF918C
:101CA0000C94DC0AEF92FF920F931F93CF93DF9374
:101CB0001F92CDB7DEB77C01FC0100811181C80104
:101CC00069830E9488306981681719F0C8010E94F1
:101CD0009030C7010F90DF91CF911F910F91FF902E
:101CE000EF900895CF92DF92EF92FF920F931F93A0
:101CF000CF93DF936C017A018B01C0E0D0E0CE1569
:101D0000DF0589F0D8016D918D01D601ED91FC912F
:101D10000190F081E02DC6010995892B11F47E0117
:101D200002C02196ECCFC701DF91CF911F910F9197
:101D3000FF90EF90DF90CF900895FC01918D828D00
:101D4000981761F0828DDF01A80FB11D5D968C910F
:101D5000928D9F5F9F73928F90E008958FEF9FEF1A
:101D60000895FC01918D828D981731F0828DE80FD6
:101D7000F11D858D90E008958FEF9FEF0895FC0190
:101D8000918D228D892F90E0805C9F4F821B91095D
:101D90008F73992708958EEA93E00E94BF0E21E089
:101DA000892B09F420E0822F0895FC01848DDF0146
:101DB000A80FB11DA35ABF4F2C91848D90E00196BE
:101DC0008F739927848FA689B7892C93A089B189AD
:101DD0008C9180648C93938D848D981306C00288B7
:101DE000F389E02D80818F7D80830895EF92FF92AB
:101DF0000F931F93CF93DF93EC0181E0888F9B8D2E
:101E00008C8D981305C0E889F989808185FD24C0EF
:101E1000F62E0B8D10E00F5F1F4F0F731127E02E72
:101E20008C8DE8120CC00FB607FCFACFE889F9894F
:101E3000808185FFF5CFCE010E94D50EF1CF8B8D2D
:101E4000FE01E80FF11DE35AFF4FF0820B8FEA8984
:101E5000FB898081806207C0EE89FF896083E88901
:101E6000F98980818064808381E090E0DF91CF9167
:101E70001F910F91FF90EF900895CF93DF93EC01A6
:101E8000888D8823C9F0EA89FB89808185FD05C09A
:101E9000A889B9898C9186FD0FC00FB607FCF5CFD4
:101EA000808185FFF2CFA889B9898C9185FFEDCF1C
:101EB000CE010E94D50EE7CFDF91CF91089580E04B
:101EC00090E0892B29F00E94CB0E81110C94000028
:101ED0000895833081F028F4813099F08230A1F0A8
:101EE00008958730A9F08830B9F08430D1F480911A
:101EF00080008F7D03C0809180008F778093800069
:101F0000089584B58F7702C084B58F7D84BD089510
:101F10008091B0008F7703C08091B0008F7D809357
:101F2000B00008953FB7F8948091A6039091A7035D
:101F3000A091A803B091A90326B5A89B05C02F3F87
:101F400019F00196A11DB11D3FBFBA2FA92F982FDF
:101F50008827820F911DA11DB11DBC01CD0142E05A
:101F6000660F771F881F991F4A95D1F70895209112
:101F7000AC033091AD032817390771F49091AA038F
:101F80008091AB03981741F0E091AA03F0E0EF597C
:101F9000FC4F808190E008958FEF9FEF08950895A2
:101FA0001F93CF93DF93DC015C962D913C915D975D
:101FB0002115310539F481E090E013969C938E93BE
:101FC00012973DC05196ED91FC91529750969C917D
:101FD0005097892F80951FB75E964C915E9741FB75
:101FE000772770F941FD6095F8944081772311F0CF
:101FF000492B01C048234083E9012197F1F748E0CC
:10200000508160FF02C0592B01C058235083E90161
:102010002197F1F76695415099F7772321F0908148
:102020008923808303C08081982B90831FBF5C9697
:102030008D919C915D970197F1F721E030E0C90106
:10204000DF91CF911F9108952091AC033091AD03A2
:102050002817390771F48091AB032091AA0390E00F
:10206000805C9F4F821B910960E470E00E94C63340
:10207000089580E090E008952091AC033091AD0385
:1020800028173907B9F49091AA038091AB039817E8
:1020900089F0E091AA03F0E0EF59FC4F8081209194
:1020A000AA0330E02F5F3F4F2F7333272093AA03FB
:1020B00090E008958FEF9FEF0895EF92FF920F93B6
:1020C0001F93DC01ED91FC9111971A960D911C91D3
:1020D0001B9718962D913C911997048CF58DE02D46
:1020E0007B0140E050E060E070E009951F910F91A6
:1020F000FF90EF9008950E94FB33611102C060E2EF
:1021000001C061E20C9437091F93CF93DF93EC0178
:10211000162F66E30E943709612F63706D8B8A8DDD
:10212000623089F16330A9F16130D1F0823011F46D
:1021300060EC01C068ECCE010E94FF0880E890E0EE
:10214000998788878A8D813019F480E890E002C0F1
:1021500080EA90E09B878A87DF91CF911F91089555
:10216000823011F460EA01C068EACE010E94FF08E3
:102170008A8D813019F480E890E002C080EA90E016
:1021800099878887E2CF823011F460E0D4CF68E08D
:10219000D2CF823011F460E6E8CF68E6E6CFAF92A6
:1021A000BF92CF92DF92EF92FF920F931F93CF9344
:1021B000DF93EC015901680128853985621773079F
:1021C0000CF05CC08A859B85481759070CF056C0F7
:1021D000FB01EA0DFB1D2E173F071CF45901A61A3F
:1021E000B70A9A012C0D3D1D821793071CF46C0150
:1021F000C41AD50A0FEF040F0C0D2FEF260F2A0D6E
:10220000CE010E94700980914B0490914C040E9471
:10221000FC08EAA1FBA190818CA5892B8083E8A111
:10222000F9A190818BA58095892380831C141D04BE
:102230009CF48501101611065CF46F2DCE010E94EE
:10224000CE086E2DCE010E94CE0801501109F2CFAA
:1022500081E0C81AD108EACFE8A1F9A190818BA545
:10226000892B8083DF91CF911F910F91FF90EF9089
:10227000DF90CF90BF90AF900C94FB08DF91CF918F
:102280001F910F91FF90EF90DF90CF90BF90AF9094
:102290000895DC01ED91FC910190F081E02D09940D
:1022A0006115710579F0FB0101900020E9F7319784
:1022B000AF01461B570BDC01ED91FC910280F381CD
:1022C000E02D099480E090E008954F925F926F9224
:1022D0007F92EF92FF920F931F93CF93DF93CDB72F
:1022E000DEB7A1970FB6F894DEBF0FBECDBF7C015D
:1022F000FA01CB0119A2223008F42AE08E010F5D09
:102300001F4F422E512C612C712CBF01A301920151
:102310000E94BD30F901CA01015011096A3014F45C
:10232000605D01C0695CD8016C93232B242B252BA5
:1023300061F7B801C7010E945011A1960FB6F89439
:10234000DEBF0FBECDBFDF91CF911F910F91FF90E8
:10235000EF907F906F905F904F9008950F931F9331
:10236000CF93DF93EC010E9450118C016FEB71E071
:10237000CE010E945011800F911FDF91CF911F91CC
:102380000F9108950C9450111F920F920FB60F9257
:1023900011242F933F934F935F936F937F938F936A
:1023A0009F93AF93BF93EF93FF938EEA93E00E94C6
:1023B000D50EFF91EF91BF91AF919F918F917F913A
:1023C0006F915F914F913F912F910F900FBE0F90A2
:1023D0001F9018951F920F920FB60F9211242F93F2
:1023E0008F939F93EF93FF93E091BE03F091BF0310
:1023F0008081E091C403F091C50382FD12C09081F9
:102400008091C7038F5F8F732091C803821751F0AB
:10241000E091C703F0E0E255FC4F958F8093C7032E
:1024200001C08081FF91EF919F918F912F910F902B
:102430000FBE0F901F901895CF93DF93282F30E099
:10244000F901ED5FF94F8491F901E15CF94FD49105
:10245000F901E55DF94FC491CC2391F081110E94FF
:10246000690FEC2FF0E0EE0FFF1FEF5DF94FA59124
:10247000B491EC91ED2381E090E021F480E002C082
:1024800080E090E0DF91CF9108951F93CF93DF9389
:10249000282F30E0F901ED5FF94F8491F901E15CFB
:1024A000F94FD491F901E55DF94FC491CC23C9F0FE
:1024B000162F81110E94690FEC2FF0E0EE0FFF1F25
:1024C000E95EF94FA591B4918FB7F894111105C049
:1024D0009C91ED2FE095E92302C0EC91ED2BEC935C
:1024E0008FBFDF91CF911F910895CF93DF9390E03D
:1024F000FC01E15CF94F2491FC01E55DF94F849109
:10250000882361F190E0880F991FFC01E750FA4F92
:10251000C591D491FC01E95EF94FA591B491611187
:1025200009C09FB7F8948881209582238883EC9115
:102530002E230BC0623061F49FB7F8943881822F4C
:10254000809583238883EC912E2B2C939FBF06C00C
:102550008FB7F894E8812E2B28838FBFDF91CF911E
:1025600008958F929F92AF92BF92CF92DF92EF9297
:10257000FF926B017C010E94920F4B015C01C11420
:10258000D104E104F104F1F00E94920FDC01CB01CF
:1025900088199909AA09BB09883E9340A105B1058C
:1025A00070F321E0C21AD108E108F10888EE880E24
:1025B00083E0981EA11CB11CC114D104E104F104F4
:1025C00019F7DDCFFF90EF90DF90CF90BF90AF90E5
:1025D0009F908F9008951F920F920FB60F92112423
:1025E0002F933F938F939F93AF93BF938091A203B9
:1025F0009091A303A091A403B091A5033091A103EE
:1026000023E0230F2D3720F40196A11DB11D05C035
:1026100026E8230F0296A11DB11D2093A1038093EC
:10262000A2039093A303A093A403B093A503809166
:10263000A6039091A703A091A803B091A9030196C6
:10264000A11DB11D8093A6039093A703A093A80397
:10265000B093A903BF91AF919F918F913F912F911B
:102660000F900FBE0F901F9018951F920F920FB6EC
:102670000F9211242F933F934F935F936F937F9308
:102680008F939F93AF93BF93EF93FF93E091AC032E
:10269000F091AD03309709F451C0968DA685B785AA
:1026A000858591FF04C09C91892329F447C09C91A2
:1026B000892309F043C0A389B4899C9185898095B9
:1026C00089238C93868997890197F1F7608D718DA5
:1026D000A685B785558538E020E0CB010197F1F755
:1026E000822F90E095958795282F4C91452309F0EE
:1026F0002068315091F7868D81FD20958091AB0344
:1027000090E001968F7399273091AA03381749F00A
:10271000A091AB03B0E0AF59BC4F2C938093AB03B7
:1027200003C0868D8160868F828D938D0197F1F72E
:10273000A389B4899C918589892B8C93FF91EF9112
:10274000BF91AF919F918F917F916F915F914F91C9
:102750003F912F910F900FBE0F901F901895E09111
:10276000AC03F091AD03E817F90769F4A389B489C4
:102770009C918589809589238C931092AD0310924A
:10278000AC0381E0089580E008952F923F924F922C
:102790005F926F927F928F929F92AF92BF92CF92F1
:1027A000DF92EF92FF920F931F93CF93DF9300D0AE
:1027B00000D000D0CDB7DEB75C014B015E834D8306
:1027C000280181E090E03C01641A750ACA019195E4
:1027D00081959109AC01440F551F5A834983180113
:1027E000CC24C394D12C522F51705B8322702C8344
:1027F000C60101972D813E81821793070CF068C0B6
:1028000077FC0CC08D819E8101979E838D83E98129
:10281000FA813296FA83E9836E0E7F1EC601880F15
:10282000991F0196680E791EFB81FF2319F12D81F6
:102830003E81220F331F2F5F3F4F240D351D87012F
:10284000A4018D819E81481B590BB6016A0D7B1D29
:1028500081E594E00E94100891012D5F3F4FA40193
:102860004C195D096D817E816A0D7B1D81E594E0C7
:102870000E9410089C81992321F12D813E81220F15
:10288000331F2F5F3F4F240D351D8701A401ED81BC
:10289000FE814E1B5F0BB5016C197D0981E594E04B
:1028A0000E94100891012D5F3F4FA4014C195D0952
:1028B000B5018D819E81681B790B81E594E00E94B2
:1028C00010089FEFC91AD90AE2E02E0E311C90CFF2
:1028D00026960FB6F894DEBF0FBECDBFDF91CF9125
:1028E0001F910F91FF90EF90DF90CF90BF90AF902E
:1028F0009F908F907F906F905F904F903F902F9020
:1029000008952F923F924F925F926F927F928F9293
:102910009F92AF92BF92CF92DF92EF92FF920F936E
:102920001F93CF93DF937C016B0166246394712C1A
:1029300000E010E0C3E0D0E09AEF892E99249A9449
:102940002EEFA22EBB24BA94842F8470582E842F8D
:102950008270482E842F8870382E4170242E0F5F8D
:102960001F4F82E0680E711CA60CB71C5520C1F0E9
:1029700024EE38EAA6014C0F5D1FB701600F711FEE
:1029800081E594E00E941C0824EE38EAA601400F7D
:10299000511FB7016C0F7D1F81E594E00E941C0858
:1029A0004420C1F024EE38EAA6014C1B5D0BB701B0
:1029B000600F711F81E594E00E941C0824EE38EA44
:1029C000A601401B510BB7016C0F7D1F81E594E000
:1029D0000E941C083320C1F024EE38EAA601400F03
:1029E000511FB7016C1B7D0B81E594E00E941C0810
:1029F00024EE38EAA6014C0F5D1FB701601B710B76
:102A000081E594E00E941C082220C1F024EE38EAFF
:102A1000A601401B510BB7016C1B7D0B81E594E0B7
:102A20000E941C0824EE38EAA6014C1B5D0BB7017E
:102A3000601B710B81E594E00E941C080C171D07B8
:102A40004CF4B7FC8CCF219782E0880E911CA80C27
:102A5000B91C85CFDF91CF911F910F91FF90EF901F
:102A6000DF90CF90BF90AF909F908F907F906F90AE
:102A70005F904F903F902F9008952F923F924F92EA
:102A80005F926F927F928F929F92AF92BF92CF92FE
:102A9000DF92EF92FF920F931F93CF93DF93CDB707
:102AA000DEB7AC970FB6F894DEBF0FBECDBF9CA7C4
:102AB0008BA73B015A014901B801DC8ACB8A261554
:102AC000370584F4892DE614F7040CF08BC1470117
:102AD0007301622E782E8B2D58016BA57CA54BA718
:102AE0008CA70DC0E216F306C4F4982D892D47017A
:102AF000E92EF82E9A2D8B2D5B01692F782F8614E5
:102B000097045CF4962D872D3401892E982E9BA571
:102B10008CA5BCA6ABA6A92EB82E6E147F0449F5D1
:102B20002BA53CA5A216B3065CF09BA58CA52A1587
:102B30003B0514F49A2D8B2DABA4BCA49BA78CA7AA
:102B40006A157B0544F04BA55CA54617570714F49E
:102B50007CA76BA7B5012BA53CA5261B370B2F5FC8
:102B60003F4F0B891C89A30181E594E00E94040872
:102B700042C1C501ABA5BCA58A1B9B0B94012619BC
:102B80003709FB01EA1BFB0BFC83EB83A70146190A
:102B9000570958874F83DB01AA19BB09BC87AB874C
:102BA000F701E819F909FE8BED8B8E149F0431F0C3
:102BB000A401415051095A8F498F02C09A8E898EC3
:102BC0006301212C312C21011F86188A198A1A8A47
:102BD000A901330F660B770B4B8F5C8F6D8F7E8F48
:102BE0002F813885032E000C440B550B2F8F38A3F3
:102BF00049A35AA3AC01990F660B770B4BA35CA3B7
:102C00006DA37EA36B817C81072E000C880B990B32
:102C10006FA378A789A79AA7A98DBA8DAC15BD0512
:102C20000CF451C06F85788989899A892B8D3C8DE8
:102C30004D8D5E8D0E949E308BA59CA5820F931FAB
:102C40009A838983C201B1012F8D38A149A15AA16C
:102C50000E949E30ABA5BCA52A0F3B1F4F8558890B
:102C600069897A898BA19CA1ADA1BEA1480F591F8A
:102C70006A1F7B1F4F87588B698B7A8B4FA158A592
:102C800069A57AA5240E351E461E571E69817A81D4
:102C90002617370734F499818A813A832983292FAB
:102CA000382F89819A81281B390B2F5F3F4F0B8961
:102CB0001C89A601BC0181E594E00E9404089FEFF5
:102CC000C91AD90AA9CFC60188199909EB85FC85CB
:102CD000E89F1001E99F300CF89F300C1124032C61
:102CE000000C44085508C601861997092B813C81C0
:102CF000289F3001299F700C389F700C1124072CDD
:102D0000000C880899084D895E89052E000C660B19
:102D1000770B4D8B5E8B6F8B788F6F817885072E4D
:102D2000000C880B990B6F83788789879A87CF016E
:102D3000092E000CAA0BBB0B8B879C87AD87BE8727
:102D4000032E000C440B550B2B833C834D835E8379
:102D5000EC14FD040CF44FC0C201B1012D893E8971
:102D60004F89588D0E949E30B501620F731F7A8380
:102D70006983C401B3012F81388549855A850E9432
:102D80009E308BA59CA5280F391F4B855C856D85D2
:102D90007E85240E351E461E571E6B817C818D81DB
:102DA0009E81660E771E881E991E89819A8128173A
:102DB000390734F499818A813A832983292F382F5E
:102DC000A981BA812A1B3B0B2F5F3F4F0B891C89BE
:102DD000A601BD0181E594E00E940408BFEFCB1A73
:102DE000DB0AB6CF4301622E782E8B2DABA4BCA498
:102DF0004BA78CA792CEAC960FB6F894DEBF0FBE51
:102E0000CDBFDF91CF911F910F91FF90EF90DF9099
:102E1000CF90BF90AF909F908F907F906F905F907A
:102E20004F903F902F900895AF92BF92CF92DF9234
:102E3000EF92FF920F931F93CF93DF936C015B018F
:102E4000EA0180EEE82EFF24FA940AE710E09B01E5
:102E500045E650E0B60181E594E00E94850605E66E
:102E600010E09E014AE750E0B50181E594E00E9440
:102E70008506960145E650E0BE0181E594E00E949A
:102E80008506DF91CF911F910F91FF90EF90DF901A
:102E9000CF90BF90AF900895AF92BF92CF92DF9244
:102EA000EF92FF920F931F93CF93DF936C015B011F
:102EB000EA0179019A01220F331F2F5F3F4FAB01C7
:102EC0004C1B5D0B8701B60181E594E00E94100860
:102ED00000E010E023E0AE01B501C6010E94C51379
:102EE000DF91CF911F910F91FF90EF90DF90CF90E6
:102EF000BF90AF900895EF92FF920F931F93CF93DF
:102F0000DF93EC017C0183E0E80EF11C04EE18EA8B
:102F100022E030E04AE050E0B70181E594E00E9411
:102F2000040822E030E04DE150E0B70181E594E093
:102F30000E9404082EE030E04DE050E0BE0181E543
:102F400094E00E941008BE01695F7F4F2EE030E0E0
:102F50004DE050E081E594E00E94100841E06DE012
:102F600070E0C7010E948114249642E06DE070E099
:102F7000CE010E94811444E06AE170E0CE010E941B
:102F8000811448E06AE170E0C701DF91CF911F91A1
:102F90000F91FF90EF900C948114CF92DF92EF92FB
:102FA000FF92CF93DF936C01990FEE08FF08F7FEB5
:102FB00016C06DE281E594E00E944911EC014427BE
:102FC0005527BA014C195D096E097F092AE081E590
:102FD00094E00E9465117C01EC0EFD1E08C02AE001
:102FE000B701A60181E594E00E9465117C016FEBB9
:102FF00071E081E594E00E9450118E0D9F1DDF91DC
:10300000CF91FF90EF90DF90CF90089510929B04A6
:1030100010929A04109299041092980410929704B6
:10302000109296048DEC90E090939D0480939C0404
:1030300090918C04963108F057C025E530E030932C
:103040009704209396042BEC30E03093990420935E
:10305000980420E930E030939B0420939A04209157
:103060006800983050F031E09E3008F430E081E0A4
:1030700001C0880F3A95EAF701C084E0822B809363
:103080006800983038F09E3040F0963148F020E0EB
:1030900030E008C02DE630E005C02BE630E002C08D
:1030A0002CE630E03093940420939304983030F46D
:1030B00081E001C0880F9A95EAF70EC0292F30E011
:1030C0009E3018F42850310902C02E50310981E099
:1030D00001C0880F2A95EAF78093950480919C049B
:1030E00090919D040197F1F780919A0490919B042F
:1030F000892B21F18091AC039091AD0324E08038BD
:103100009207E1F0009711F00E94AF1380919E04A6
:103110008E7F80939E041092AB031092AA0380E8E6
:1031200094E09093AD038093AC03E0919304F0910D
:103130009404908180919504892B80830895CF9287
:10314000DF92EF92FF920F931F93CF93DF936B0168
:10315000770FEE08FF08F7FE1BC0EC016DE20E943E
:1031600049118C0144275527BA014C195D096E0994
:103170007F092AE0CE010E946511800F911FDF9127
:10318000CF911F910F91FF90EF90DF90CF90089516
:103190002AE0B701A601DF91CF911F910F91FF9017
:1031A000EF90DF90CF900C946511CF93DF93EC01FB
:1031B00061E085E00E947512209711F460E004C080
:1031C000CF3FD10531F461E085E0DF91CF910C94E0
:1031D0004512E8E0F6E0E491E330F9F048F4E1303C
:1031E000B9F0E230A1F584B5806284BDC8BD34C0B9
:1031F000E730E9F0E83019F1E43049F580918000DA
:10320000806280938000D0938B00C0938A0024C09A
:1032100084B5806884BDC7BD1FC080918000806870
:1032200080938000D0938900C093880015C080915E
:10323000B00080688093B000C093B3000DC080914F
:10324000B00080628093B000C093B40005C0C03865
:10325000D1050CF0B8CFB2CFDF91CF910895CF92C6
:10326000DF92EF92FF920F931F93CF93DF93EC01C6
:103270002196FC011491112309F437C0FE016491D9
:1032800081E594E00E9437096E01F2E0CF0ED11C77
:10329000FE013196C4910C2F0078CF777601DC2F98
:1032A000D15050F0F701649181E594E00E94FF084D
:1032B000FFEFEF1AFF0AF4CFC6018C0F911DEC014E
:1032C000002389F07C019FEFE91AF90AFE0164915D
:1032D00070E06F3F710511F464EF71E080E090E001
:1032E0000E94B112E7011150C6CFDF91CF911F911B
:1032F0000F91FF90EF90DF90CF9008952F923F9223
:103300004F925F926F927F928F929F92AF92BF92F5
:10331000CF92DF92EF92FF920F931F93CF93DF93A1
:1033200000D000D0CDB7DEB78C017B015C834B832E
:1033300081E090E05C01A41AB50ACA0191958195DB
:1033400091091C01220C331C460F571F20EE3FEF42
:10335000B80181E594E00E941C08A7012B813C8103
:10336000421B530B20EE3FEFB80181E594E00E9431
:103370001C086B817C81600F711F20EE3FEFA7015D
:1033800081E594E00E941C08B8018B819C81681B38
:10339000790B20EE3FEFA70181E594E00E941C0825
:1033A000C12CD12CE1E0F0E0FA83E9832B813C8150
:1033B000C216D3060CF076C0B7FC0BC02B813C8143
:1033C000215031093C832B8332E0230E311CA20CA7
:1033D000B31C8FEFC81AD80AE981FA813296FA83B2
:1033E000E983AE0EBF1E3601600E711E20EE3FEF68
:1033F0008B809C808E0C9F1CA401B30181E594E01E
:103400000E941C0828014C185D0820EE3FEFA40123
:10341000B20181E594E00E941C0820EE3FEF4701D5
:103420008B819C81881A990AA401B30181E594E0FB
:103430000E941C0820EE3FEFA401B20181E594E058
:103440000E941C0846018E0C9F1C20EE3FEFA40139
:103450006B807C80600E711EB30181E594E00E9458
:103460001C0820EE3FEFA4012801EB81FC814E1ADD
:103470005F0AB20181E594E00E941C0847018C18A4
:103480009D0820EE3FEFA401B30181E594E00E9486
:103490001C0820EE3FEFA401B20181E594E00E94F8
:1034A0001C0884CF0F900F900F900F90DF91CF9159
:1034B0001F910F91FF90EF90DF90CF90BF90AF9052
:1034C0009F908F907F906F905F904F903F902F9044
:1034D0000895CF93DF9300D000D000D0CDB7DEB7F2
:1034E000789484B5826084BD84B5816084BD85B5DF
:1034F000826085BD85B5816085BD80916E008160EB
:1035000080936E0010928100809181008260809390
:103510008100809181008160809381008091800092
:103520008160809380008091B10084608093B100BD
:103530008091B00081608093B00080917A008460B7
:1035400080937A0080917A00826080937A008091E3
:103550007A00816080937A0080917A0080688093FD
:103560007A001092C10060E084E00E94751260E071
:1035700087E00E94751260E086E00E94751261E0AB
:1035800085E00E947512E091BE03F091BF0382E0D6
:103590008083E091BA03F091BB031082E091BC03F9
:1035A000F091BD0387E680831092C603E091C203C9
:1035B000F091C30386E08083E091C003F091C103E2
:1035C000808180618083E091C003F091C10380819C
:1035D00088608083E091C003F091C103808180689E
:1035E0008083E091C003F091C10380818F7D80834F
:1035F00064E170E080E090E00E94B1126DE671E05D
:103600008EEA93E00E94AE110E94061864E170E019
:1036100080E090E00E94B11264E671E08EEA93E0EF
:103620000E94AE1164E170E080E090E00E94B1126F
:103630000E94E20A0E94C50AB2E02B2E312C84E0DF
:103640000E941C12082F80935B0386E00E941C12CC
:10365000182F8093430387E00E941C1280935A0323
:10366000013009F063C0113009F060C060E871E01A
:103670008EEA93E00E94C2110E94DC0A2DE030E045
:1036800030935E0420935D0480E290E090936004A8
:1036900080935F041093650420E038EF3093640456
:1036A00020936304309362042093610464E971E021
:1036B00081E594E00E94C211609150041A8219823F
:1036C000CE0101960E94520E60914F0481E090E07D
:1036D0009A838983CE0101960E94520E60914E0416
:1036E0003A822982CE0101960E94520E60914D04C9
:1036F00023E030E03A832983CE0101960E94520EE6
:1037000068EE73E080E090E00E94B11264EA71E03C
:1037100081E594E00E94C21168EE73E080E090E0E1
:103720000E94B1120E94DC0A10931B0180915B037E
:10373000811119C0809143038130A9F480914E0416
:103740008F5F833019F080934E0402C010924E04B4
:103750000E94DC0A64E670E080E090E00E94B11212
:1037600081E080931B0180915B03813009F04DC0A3
:1037700080915A03811149C0809150048A508B3046
:1037800008F483ED809350046DEA71E08EEA93E0D3
:103790000E94C2114091500450E060E070E02AE0C5
:1037A0008EEA93E00E9465116FEB71E08EEA93E080
:1037B0000E9450118091500490E00E94D5182091F1
:1037C0005004269530E0A0EEEA2EFF24FA940FE78D
:1037D00010E04FE750E060E070E081E594E00E9487
:1037E000850662E370E080E090E00E94B1122091D3
:1037F0005004269530E0E12CF12C4FE750E060E0DA
:1038000070E081E594E00E94850680915B03813041
:1038100009F04CC080915A03813009F047C0809173
:103820004F048A5009F487E980934F0462EC71E0F9
:103830008EEA93E00E94C21140914F0450E060E094
:1038400070E02AE08EEA93E00E9465116FEB71E070
:103850008EEA93E00E94501180914F0490E00E9404
:10386000D51820914F04269530E0FFE1EF2EF12C82
:103870000FE710E04FE750E060E070E081E594E092
:103880000E94850662E370E080E090E00E94B11241
:1038900020914F04269530E0E12CF12C4FE750E0C9
:1038A00060E070E081E594E00E94850680915A0313
:1038B000811103C08091500404C0813029F48091AB
:1038C0004F0490E00E94D51880915B0381110C9405
:1038D000572E8091430381110C94572E80E894E079
:1038E0000E9424101816190614F00C94142E80E867
:1038F00094E00E943C106C0162E070E080E090E097
:103900000E94B1128091410390914203039719F4F0
:1039100031E0C31AD108C114D10439F467E872E068
:103920008EEA93E00E94C21104C0D7FE02C00C943C
:10393000572E80913F03909140038F30910514F0F2
:103940000C94572E01969093400380933F0366EDAD
:1039500071E08EEA93E00E94C211B6018EEA93E014
:103960000E949F1862E070E080E090E00E94B11237
:1039700080913F0390914003019709F0C2C280916A
:103980005803909159038C159D0509F4BAC2D09241
:103990001A01C0921901D0925903C092580385E5CB
:1039A000C816D10434F085E590E090931A01809315
:1039B000190180914E0481115DC0E12CF12C0AE0C7
:1039C00010E02DE030E04FE150E06FE170E081E584
:1039D00094E00E94CF10A0901901B0901A0126E542
:1039E00030E02A193B09B5016A5B7F4F4FE150E097
:1039F00081E594E00E94CF109AE0A916B1046CF41E
:103A000087E290E090935E0480935D0420E230E0D2
:103A10003093600420935F040CC081E290E09093A7
:103A20005E0480935D0480E290E090936004809354
:103A30005F0481E08093650480EE97E090936404D6
:103A4000809363049093620480936104C5010E9493
:103A5000CD172091190130911A01E12CE8EFFE2ECB
:103A600008E010E04FE150E067E470E081E594E0A9
:103A70000E94CF1080914E04813009F02FC1E12CBB
:103A8000F12C06E110E022E230E048E250E066E08E
:103A900070E081E594E00E94CF108091190190912F
:103AA0001A018A3091051CF428E130E002C026E0BA
:103AB00030E030935E0420935D0428E230E03093E0
:103AC000600420935F0423E02093650420EE37E038
:103AD0003093640420936304309362042093610460
:103AE00024E6289FB001299F700D112481E594E000
:103AF0000E949F188091190190911A0105971CF05E
:103B000060EE77E002C060E070E082E090E00E944A
:103B10003B2F8091190190911A010A971CF060EED9
:103B200077E002C060E070E08CE090E00E943B2F04
:103B30008091190190911A010F971CF060EE77E0C7
:103B400002C060E070E086E190E00E943B2F80912F
:103B5000190190911A0144971CF060EE77E002C0C1
:103B600060E070E080E290E00E943B2F80911901BC
:103B700090911A0149971CF060EE77E002C060E076
:103B800070E08AE290E00E943B2F809119019091B1
:103B90001A014E971CF060EE7FEF02C060E070E00B
:103BA00084E390E00E943B2F8091190190911A01CB
:103BB00083971CF060EE7FEF02C060E070E08EE360
:103BC00090E00E943B2F8091190190911A018897F3
:103BD0001CF060EE7FEF02C060E070E088E490E0EF
:103BE0000E943B2F8091190190911A018D971CF032
:103BF00060EA7DEF02C060E070E082E590E00E9444
:103C00003B2F8091190190911A01C2971CF060EA34
:103C10007DEF02C060E070E08CE590E00E943B2FF9
:103C20008091190190911A01C7971CF060E078EF1C
:103C300002C060E070E086E690E00E943B2F809139
:103C4000190190911A01CC971CF060E078EF02C046
:103C500060E070E080E790E00E943B2F80911901C6
:103C600090911A01813491051CF066EB7BE802C04B
:103C700060E070E08AE790E00E943B2F809119019C
:103C800090911A01863491051CF066EB7BE802C026
:103C900060E070E084E890E00E943B2F8091190181
:103CA00090911A018B3491051CF06FEF7FEF02C0E9
:103CB00060E070E08EE890E00E943B2F8091190157
:103CC00090911A01803591051CF06FEF7FEF02C0D3
:103CD00060E070E088E990E00E943B2F80914E0404
:103CE000823009F00EC10091170110911801209146
:103CF000150130911601E12CF12C4BE450E060E508
:103D000070E081E594E00E94850620EE3FEF46E0FA
:103D100050E060E570E080E590E00E944C1770EEA6
:103D2000E72EFF24FA940EE010E027E130E04FE4A4
:103D300050E069E370E081E594E00E94CF1020E05C
:103D400030E041E050E06EE470E080E590E00E94F9
:103D50004C17B6010D2C000C880B990B0E940F32EA
:103D60004B015C0120E030E048EA52E40E94FE3260
:103D7000181634F4812C912C6AEAA62E62E4B62E31
:103D8000A5019401C501B4010E94EF309B01AC0173
:103D900060E070E084E393E40E94EE309B01AC01AC
:103DA00060E070E084E393E40E9465319B01AC0124
:103DB00067E876E189E490E40E9465314B015C019B
:103DC0000E9460312B013C01C501B4010E94703397
:103DD0004B015C0120E030E044E752E4C301B20152
:103DE0000E9403330E94D731605B7F4F70931601AE
:103DF0006093150120E030E044E752E4C501B401CE
:103E00000E9403330E94D73120E530E0C901861BB0
:103E1000970B90931801809317018091190190914D
:103E20001A018997449750F420E030E047E050E0D1
:103E300068E270E080E590E00E944C1780911901E3
:103E400090911A010091170110911801209115010C
:103E500030911601CD97F4F0E12C58EFF52E4BE49C
:103E600050E060E570E081E594E00E94850620E086
:103E700038EF46E050E068E270E080E590E00E94B4
:103E80004C1747E050E068E270E080E590E00E9467
:103E90007E190CC040EEE42EFF24FA944BE450E06F
:103EA00060E570E081E594E00E948506609119016B
:103EB00070911A016A3071051CF486E490E002C02A
:103EC0008AE390E090935E0480935D048FE490E039
:103ED0009093600480935F0482E080936504109265
:103EE000640410926304109262041092610481E5EC
:103EF00094E00E949F186FEF71E081E594E00E94CA
:103F0000C21180913F0390914003029709F0C7C10D
:103F100080915603909157038C159D0509F4BFC1FC
:103F2000D0921401C0921301D0925703C09256034D
:103F300080914E0481117BC0E12CF12C0AE010E04D
:103F400024E130E04EE250E06FE170E081E594E082
:103F50000E94CF10B6010D2C000C880B990B0E940B
:103F60000F3223EC35EF48EA5EE30E9403332B0166
:103F70003C019B01AC0160E070E08CEA92E40E949D
:103F8000EE300E94D7314B015C0120E030E04CE87C
:103F900052E4C301B2010E94EF300E94D73109E020
:103FA00010E094014FE250E081E594E00E94CF10D0
:103FB00080EE9FEF90936404809363049093620477
:103FC0008093610481E290E090935E0480935D04AD
:103FD0008FE290E09093600480935F0481E080938F
:103FE0006504B60181E594E00E949F186091130179
:103FF00070911401072E000C880B990B0E940F3250
:1040000023EC35EF48EA5EE30E9403330E94D73188
:1040100020EEE22EFF24FA9408E010E09B014FE22C
:1040200050E067E470E081E594E00E94CF10809159
:104030004E04882309F433C12091550330E02C5FEE
:104040003F4FE12CF12C03E610E048E750E065E13A
:1040500070E081E594E00E9485062091550330E0F0
:104060002C5F3F4F48E750E066E170E081E594E067
:104070000E9485062091550330E02C5F3F4F48E7B2
:1040800050E067E170E081E594E00E9485062091B0
:10409000130130911401C90167E070E00E94C6333A
:1040A000609355032333310554F577279B012C5F2B
:1040B0003F4FEE24EA9497E0F92E48E750E065E19F
:1040C00070E081E594E00E9485062091550330E080
:1040D0002C5F3F4F48E750E066E170E081E594E0F7
:1040E0000E9485062091550330E02C5F3F4F48E742
:1040F00050E067E170E081E594E00E9485068091E0
:10410000130190911401C397C29760F52091550354
:1041100030E02C5F3F4FE12C88EFF82E03E610E0F3
:1041200048E750E065E170E081E594E00E94850693
:104130002091550330E02C5F3F4F48E750E066E1A7
:1041400070E081E594E00E9485062091550330E0FF
:104150002C5F3F4F48E750E067E170E081E594E075
:104160000E94850680911301909114018556910952
:10417000C29768F52091550330E02C5F3F4F00EE69
:10418000E02E07E0F02E03E610E048E750E065E19E
:1041900070E081E594E00E9485062091550330E0AF
:1041A0002C5F3F4F48E750E066E170E081E594E026
:1041B0000E9485062091550330E02C5F3F4F48E771
:1041C00050E067E170E081E594E00E94850680910F
:1041D00013019091140187599109C29768F52091B4
:1041E000550330E02C5F3F4F10EAE12E1DEFF12E1A
:1041F00003E610E048E750E065E170E081E594E017
:104200000E9485062091550330E02C5F3F4F48E720
:1042100050E066E170E081E594E00E94850620911F
:10422000550330E02C5F3F4F48E750E067E170E016
:1042300081E594E00E94850680911301909114011C
:10424000893C910564F12091550330E02C5F3F4F8C
:10425000EE24EA94FE2C03E610E048E750E065E126
:1042600070E081E594E00E9485062091550330E0DE
:104270002C5F3F4F48E750E066E170E081E594E055
:104280000E9485062091550330E02C5F3F4F48E7A0
:1042900050E067E170E081E594E00E94850680913E
:1042A0003F0390914003039709F02DC18091530380
:1042B000909154038C159D0509F425C1D0921201EB
:1042C000C0921101D0925403C092530395E6C916CF
:1042D000D10434F084E690E09093120180931101B0
:1042E00080914E0481117BC080EE9FEF9093640417
:1042F000809363049093620480936104E12CF12C19
:104300000AE010E024E130E041E050E06FE170E0CD
:1043100081E594E00E94CF102091110130911201AB
:104320003C832B83B901330F880B990B0E940F320A
:104330002DE33AE047E55FE30E9403334B015C0164
:104340009B01AC0160E070E08CEA92E40E94EE30E8
:104350000E94D7312B013C0120E030E04CE852E4D0
:10436000C501B4010E94EF300E94D731920141E0B3
:1043700050E081E594E00E94CF1081E290E09093BC
:104380005E0480935D043092600420925F0481E0BB
:10439000809365048B819C810E94CD1760911101EF
:1043A00070911201072E000C880B990B0E940F329E
:1043B0002DE33AE047E55FE30E9403330E94D731E3
:1043C000EE24EA94A7E0FA2E08E010E09B0142E018
:1043D00050E067E470E081E594E00E94CF108091A6
:1043E0004E04813009F08FC0A0901101B0901201ED
:1043F000B5010B2C000C880B990B0E940F3221EE9B
:104400003AE744E15FE30E9403332B013C019B0147
:10441000AC0160E070E080E792E40E94EE300E9420
:10442000D7316B837C838D839E8320E030E044E131
:1044300052E4C301B2010E94EF300E94D731E12C57
:10444000F12C0AE010E02B813C814AE450E081E548
:1044500094E00E94CF10C301B2010E94D731EE2434
:10446000EA94F7E0FF2E08E010E09B014BE450E0F7
:1044700066E270E081E594E00E94CF108FEF97E054
:104480009093640480936304909362048093610426
:104490003AE0A316B104BCF088E190E090935E048A
:1044A00080935D048BE490E09093600480935F04BC
:1044B00024E6A216B1049CF025E130E030935E04BE
:1044C00020935D0408C08EE190E090935E04809399
:1044D0005D048BE490E09093600480935F0481E03E
:1044E00080936504E12CF12C09E010E020E130E03C
:1044F0004BE450E066E170E081E594E00E94CF106B
:10450000C5010E94CD1780913F039091400304970D
:1045100009F059C180915103909152038C159D056A
:1045200009F451C1D0921001C0920F01D0925203F0
:10453000C092510380914E04811177C0E12CF12C7F
:1045400009E010E024E130E04DE350E06FE170E07D
:1045500081E594E00E94CF10B6010D2C000C880B71
:10456000990B0E940F322DE33AE047E55FE30E948A
:1045700003332B013C019B01AC0160E070E08CEA4D
:1045800092E40E94EE300E94D7314B015C0120E0A2
:1045900030E04CE852E4C301B2010E94EF300E94C7
:1045A000D73194014EE350E081E594E00E94CF10B2
:1045B00080EE9FEF90936404809363049093620471
:1045C0008093610481E290E090935E0480935D04A7
:1045D0008EE390E09093600480935F0481E0809389
:1045E0006504C6010E94CD1760910F017091100102
:1045F000072E000C880B990B0E940F322DE33AE036
:1046000047E55FE30E9403330E94D731EE24EA942A
:10461000E7E0FE2E08E010E09B014EE350E067E487
:1046200070E081E594E00E94CF1080914E048150AB
:10463000823008F0C8C02091500330E028583F4F26
:10464000E12CF12C03E610E048E750E067E870E069
:1046500081E594E00E9485062091500330E02858BF
:104660003F4F48E750E068E870E081E594E00E9441
:1046700085062091500330E028583F4F48E750E02E
:1046800069E870E081E594E00E94850620910F01C1
:1046900030911001C90163E070E00E94C63360935D
:1046A00050032F3131054CF577279B0128583F4F98
:1046B000E12C78EFF72E48E750E067E870E081E5FD
:1046C00094E00E9485062091500330E028583F4F27
:1046D00048E750E068E870E081E594E00E948506D4
:1046E0002091500330E028583F4F48E750E069E8F8
:1046F00070E081E594E00E94850680910F01909121
:1047000010014F974E9760F52091500330E02858E4
:104710003F4FEE24EA94FE2C03E610E048E750E019
:1047200067E870E081E594E00E94850620915003DF
:1047300030E028583F4F48E750E068E870E081E5F6
:1047400094E00E9485062091500330E028583F4FA6
:1047500048E750E069E870E081E594E00E94850652
:1047600080910F0190911001CD976CF12091500331
:1047700030E028583F4F50EEE52E57E0F52E03E687
:1047800010E048E750E067E870E081E594E00E94BF
:1047900085062091500330E028583F4F48E750E00D
:1047A00068E870E081E594E00E948506209150035E
:1047B00030E028583F4F48E750E069E870E081E575
:1047C00094E00E94850680913F03909140030597F5
:1047D00009F01BC180914E0390914F038C159D05EC
:1047E00009F413C1D0920E01C0920D01D0924F0373
:1047F000C0924E0381E08093650480914E04811144
:104800006CC0A0903E03B12C25E530E0D6010E949B
:10481000DA33950128583F4F032E000C440B550BFB
:104820000E949E30263531052CF430930C012093E4
:104830000B0106C086E590E090930C0180930B017C
:10484000E12CF12C09E010E024E130E04CE450E0F0
:104850006FE170E081E594E00E94CF1060910B0160
:1048600070910C0126E530E0261B370B6A5B7F4F09
:104870004DE450E081E594E00E94CF1080EE9FEF80
:104880009093640480936304909362048093610422
:1048900020E230E030935E0420935D048DE490E0EC
:1048A0009093600480935F04B6016A197B0981E5E7
:1048B00094E00E949F1820910B0130910C0140EA76
:1048C000E42E4DEFF42E08E010E04DE450E067E4F4
:1048D00070E081E594E00E94CF1080914E0488231F
:1048E00009F493C080914C0390914D03892B09F0FA
:1048F0008CC080913E03A0900D01B0900E01A81ACB
:10490000B10834E6A316B104D4F080E890E09093A7
:104910005E0480935D0482E490E090936004809351
:104920005F0480EE9FEF9093640480936304909300
:10493000620480936104E12C28EFF22E57C0C50178
:104940008A5591090A97C8F483E890E090935E0431
:1049500080935D0482E490E09093600480935F0410
:104960001092640410926304109262041092610425
:1049700090EEE92EFF24FA9439C0C50186549109BE
:104980004497D0F483E890E090935E0480935D04B4
:1049900082E490E09093600480935F0480EE9FEF48
:1049A0009093640480936304909362048093610401
:1049B0008FE1E82EF12C1AC083E890E090935E041A
:1049C00080935D0482E490E09093600480935F04A0
:1049D0008FE190E090936404809363049093620469
:1049E00080936104EE24EA9407E0F02E0BE010E0DF
:1049F00025E130E040E450E06EE770E081E594E0CE
:104A00000E94CF10C5010E94CD1780913F03909165
:104A10004003069709F083C080914A0390914B03AD
:104A20008C159D0509F47BC0D0920A01C092090142
:104A3000D0924B03C0924A0380914E0481116FC003
:104A400025E530E0D6010E94DA3320913E0330E0C4
:104A500028583F4F032E000C440B550B0E949E30EC
:104A6000263531052CF4309308012093070106C048
:104A700086E590E09093080180930701E12CF12CEA
:104A800009E010E024E130E04BE550E06FE170E038
:104A900081E594E00E94CF106091070170910801B8
:104AA00027E530E0261B370B6A5B7F4F4CE550E073
:104AB00081E594E00E94CF1080EE9FEF9093640414
:104AC00080936304909362048093610480E290E099
:104AD00090935E0480935D048CE590E09093600475
:104AE00080935F0481E08093650480910601B601A4
:104AF000681B710981E594E00E949F1820910701CD
:104B000030910801EE24EA94FE2C08E010E04CE518
:104B100050E067E470E081E594E00E94CF1080915E
:104B20003F0390914003079709F087C080914803A5
:104B3000909149038C159D0509F47FC092E0C91638
:104B4000D1040CF47AC080914E04811176C0D092C9
:104B50000501C0920401D0924903C0924803E12CA0
:104B6000F12C0AE010E02AE130E04AE650E06FE183
:104B700070E081E594E00E94CF1020E230E03093B5
:104B80005E0420935D048BE690E090936004809334
:104B90005F0480EE9FEF909364048093630490938E
:104BA00062048093610481E080936504C6010E94E1
:104BB000CD176091040170910501072E000C880B40
:104BC000990B0E940F3228EB3EE145E05FE30E9423
:104BD00003334B015C019B01AC0160E070E08CEAA7
:104BE00092E40E94EE300E94D7312B013C0120E07C
:104BF00030E04CE852E4C501B4010E94EF300E945D
:104C0000D73109E010E092014BE650E081E594E0F5
:104C10000E94CF10C501B4010E94D731B0EEEB2E37
:104C2000FF24FA9408E010E09B014BE650E067E4B3
:104C300070E081E594E00E94CF1080913F03909155
:104C40004003089709F092C180914C0390914D0365
:104C5000892B09F08BC1B601DD0C880B990B0E94E2
:104C60000F324B015C019B01AC01609144037091D8
:104C7000450380914603909147030E945B3188234E
:104C800009F474C18092000190920101A092020186
:104C9000B09203018092440390924503A092460390
:104CA000B092470381E08093650480914E048111A6
:104CB000C9C0E12CF12C0AE010E02AE130E040E12B
:104CC00050E06FE170E081E594E00E94CF1080E257
:104CD00090E090935E0480935D0481E190E0909376
:104CE000600480935F0480EE9FEF90936404809350
:104CF0006304909362048093610420E030E040E21A
:104D000051E4C501B4010E9465310E94652E4090B6
:104D1000000150900101609002017090030120E0B9
:104D200030E040EC5FE3C301B2010E94653120E056
:104D300030E040E252E40E94EE304B015C019B0106
:104D4000AC0160E070E08CEA92E40E94EE300E94D8
:104D5000D7316B837C838D839E8320E030E04CE8E9
:104D600052E4C501B4010E94EF300E94D73109E03E
:104D700010E02B813C8141E150E081E594E00E940C
:104D8000CF1020E030E046EE52E4C301B2010E94B1
:104D90005B3187FF13C0C501B4010E94D731A0EA7F
:104DA000EA2EADEFFA2E08E010E09B0141E150E061
:104DB00067E470E081E594E00E94CF1020E030E0ED
:104DC00044EE52E4C301B2010E94FE321816ECF424
:104DD00020E030E041E153E4C301B2010E945B31C5
:104DE00087FF13C0C501B4010E94D731F0EEEF2E4A
:104DF000F7E0FF2E08E010E09B0141E150E067E49E
:104E000070E081E594E00E94CF1020E030E040E1C6
:104E100053E4C301B2010E94FE3218169CF4C5018E
:104E2000B4010E94D731E0EAEE2EEDEFFE2E08E04D
:104E300010E09B0141E150E067E470E081E594E01F
:104E40000E94CF1080914E04882309F48FC081E422
:104E500090E090935E0480935D0480E790E09093EF
:104E6000600480935F048090000190900101A09005
:104E70000201B090030120E030E040EF52E4C501B0
:104E8000B4010E94FE321816C4F470EEE72E77E0EB
:104E9000F72E0FE010E02EE130E04CE650E061E448
:104EA00070E081E594E00E94CF10109264041092AB
:104EB0006304109262041092610420E030E044EE3A
:104EC00052E4C501B4010E94FE32181614F520E028
:104ED00030E042EF52E4C501B4010E945B3187FF2C
:104EE00018C060EEE62EFF24FA940FE010E02EE1E9
:104EF00030E04CE650E061E470E081E594E00E942F
:104F0000CF10109264041092630410926204109205
:104F1000610420E030E046EE52E4C501B4010E9495
:104F20005B3187FF19C0E12C58EFF52E0FE010E040
:104F30002EE130E04CE650E061E470E081E594E081
:104F40000E94CF1080EE9FEF9093640480936304DF
:104F5000909362048093610420E030E040E251E4E9
:104F6000C501B4010E9465310E94652E10911B019C
:104F7000113009F034C680914E0481508E3F08F400
:104F8000CDC124E130E030935E0420935D04309382
:104F9000600420935F04109365048FE190E0909388
:104FA00064048093630490936204809361046BEDC6
:104FB00071E081E594E00E94AE1168EC70E080E061
:104FC00090E00E94B1120E94DC0A80EE97E090937C
:104FD000640480936304909362048093610430922C
:104FE0005E0420925D043092600420925F0410936E
:104FF000650464EE71E081E594E00E94AE1121E267
:10500000C22ED12CD0925E04C0925D043092600416
:1050100020925F0468EE71E081E594E00E94AE1199
:105020003FE1E32EF12C0CE010E02FE930E040E00E
:1050300050E060E070E081E594E00E94260628E2FE
:1050400030E040E050E06EE170E081E594E00E94E5
:10505000260630925E0420925D0401E110E0109378
:10506000600400935F046EEE71E081E594E00E94BD
:10507000AE11D0925E04C0925D0410936004009360
:105080005F0462EF71E081E594E00E94AE110CE0F4
:1050900010E02FE930E04FE050E060E070E081E5A3
:1050A00094E00E94260628E230E04FE050E06EE1F6
:1050B00070E081E594E00E94260630925E04209222
:1050C0005D0480E290E09093600480935F0469EF58
:1050D00071E081E594E00E94AE11D0925E04C0922E
:1050E0005D0420E230E03093600420935F046DEFB4
:1050F00071E081E594E00E94AE112FE930E04EE1CD
:1051000050E060E070E081E594E00E94260628E22D
:1051100030E04EE150E06EE170E081E594E00E9405
:10512000260630925E0420925D040FE210E0109398
:10513000600400935F0462E072E081E594E00E9405
:10514000AE11D0925E04C0925D041093600400938F
:105150005F0466E072E081E594E00E94AE110CE02D
:1051600010E02FE930E04DE250E060E070E081E5D2
:1051700094E00E94260628E230E04DE250E06EE125
:1051800070E081E594E00E94260630925E04209251
:105190005D040EE310E01093600400935F046AE086
:1051A00072E081E594E00E94AE11D0925E04C0925C
:1051B0005D041093600400935F040CE010E02FE99D
:1051C00030E04CE350E060E070E081E594E00E9464
:1051D000260628E230E04CE350E06EE170E081E525
:1051E00094E00E94260630925E0420925D040DE455
:1051F00010E01093600400935F046EE072E081E5BC
:1052000094E00E94AE11D0925E04C0925D041093AF
:10521000600400935F040CE010E02FE930E04BE401
:1052200050E060E070E081E594E00E94260628E20C
:1052300030E04BE450E06EE170E081E594E00E94E4
:10524000260630925E0420925D040CE510E0109377
:10525000600400935F0464E172E081E594E00E94E1
:10526000AE11D0925E04C0925D041093600400936E
:105270005F040CE010E02FE930E04AE550E060E028
:1052800070E081E594E00E94260628E230E04AE5DD
:1052900050E06EE170E081E594E00E9426063092D5
:1052A0005E0420925D044BE6C42ED12CD0926004A3
:1052B000C0925F0468E172E081E594E00E94AE1163
:1052C0002FE930E049E650E060E070E081E594E0ED
:1052D0000E94260628E230E049E650E06EE170E0E8
:1052E00081E594E00E94260680E290E090935E04BF
:1052F00080935D04D0926004C0925F0480EE9FEFC3
:105300009093640480936304909362048093610497
:1053100062EE71E081E594E00E94AE11D0904E04FF
:1053200091E0D91228C224E130E030935E0420934A
:105330005D043093600420935F04D09265040FE114
:1053400010E01093640400936304109362040093CC
:1053500061046CE172E081E594E00E94AE1164EFBB
:1053600071E080E090E00E94B1120E94DC0AD092CD
:105370006504109364040093630410936204009323
:1053800061048BE090E090935E0480935D0481E083
:1053900090E09093600480935F0463E272E081E5A3
:1053A00094E00E94C21110935E0400935D0421E01A
:1053B00030E03093600420935F0466E372E081E59F
:1053C00094E00E94C21183E390E090935E04809386
:1053D0005D0481E090E09093600480935F0465E257
:1053E00072E081E594E00E94C21187E490E090931E
:1053F0005E0480935D0421E030E0309360042093EC
:105400005F0467E272E081E594E00E94C2118BE5DF
:1054100090E090935E0480935D0481E090E090932F
:10542000600480935F0463E972E081E594E00E9488
:10543000C2118FE690E090935E0480935D0421E0BA
:1054400030E03093600420935F0469E272E081E50C
:1054500094E00E94C21183E890E090935E048093F0
:105460005D0481E090E09093600480935F046BE2C0
:1054700072E081E594E00E94C21187E990E0909388
:105480005E0480935D0421E030E03093600420935B
:105490005F046DE272E081E594E00E94C21180E059
:1054A00090E00E947B178AE090E00E947B1784E1E5
:1054B00090E00E947B178EE190E00E947B1788E2CB
:1054C00090E00E947B1782E390E00E947B178CE3C0
:1054D00090E00E947B1786E490E00E947B1780E5B5
:1054E00090E00E947B178AE590E00E947B1784E69B
:1054F00090E00E947B178EE690E00E947B1788E781
:1055000090E00E947B1782E890E00E947B178CE875
:1055100090E00E947B1786E990E00E947B17FFE1F4
:10552000EF2EF12C0CE010E022E630E049E450E0F0
:1055300060E070E081E594E00E9426068FEF97E03E
:105540009093640480936304909362048093610455
:1055500083E090E090935E0480935D048BE490E0A0
:105560009093600480935F04D092650464EE71E0D0
:1055700081E594E00E94AE11A0EEEA2EFF24FA9499
:1055800001E110E020E230E04BE650E060E470E042
:1055900081E594E00E94260603E010E024E030E07C
:1055A00048E650E064E470E081E594E00E9426065D
:1055B00024E030E048E650E068E570E081E594E002
:1055C0000E9426062FE130E04CE050E065E470E0F8
:1055D00088E890E00E944C17BFE1CB2ED12C1FE34E
:1055E000E12EF12C01E910E02DE230E048E850E036
:1055F0006FE370E08FE790E00E943D154DE950E0C9
:1056000068E870E083E790E00E941417C12CD12C69
:1056100005E6E02EF12C0BE910E028E730E048E841
:1056200050E065E670E084E790E00E943D1541E2BD
:1056300050E06EE770E088E890E00E947E19E12C6F
:10564000F12C06E210E02FE030E041E650E064E6A5
:1056500070E081E594E00E94CF1008E010E02AE0BD
:1056600030E041E650E06EE970E081E594E00E94B0
:10567000CF108DE890E090935E0480935D0488E7FE
:10568000A82EB12CB0926004A0925F046AE072E090
:1056900081E594E00E94C2114BE250E066E170E0C7
:1056A00081E090E00E94141795E6E92EF12C0AE2C1
:1056B00010E028E730E046E150E065E670E082E087
:1056C00090E00E943D1541E250E06EE770E086E117
:1056D00090E00E947E19E12CF12C06E210E02FE010
:1056E00030E043E650E06CE270E081E594E00E9437
:1056F000CF1003E010E021E030E043E650E060E04E
:1057000070E081E594E00E94CF1020EE3FEF4FE57E
:1057100050E06BE170E081E594E00E94660A20EEC3
:105720003FEF4FE550E061E170E081E594E00E94D9
:10573000660A20EE3FEF41E650E06AE070E081E566
:1057400094E00E94660A20EE3FEF41E650E062E2FC
:1057500070E081E594E00E94660A10925E04109267
:105760005D04B0926004A0925F0462E072E081E5A3
:1057700094E00E94C21180914E04823009F00DC263
:1057800024E130E030935E0420935D0430936004A4
:1057900020935F0481E0809365048FE1C82ED12CB3
:1057A000D0926404C0926304D0926204C0926104F7
:1057B0006FE272E081E594E00E94AE1164EF71E067
:1057C00080E090E00E94B1120E94DC0A1092640412
:1057D0001092630410926204109261042FE130E091
:1057E0004FE450E060E570E080E590E00E944C17E7
:1057F00020EE37E04DE450E060E570E080E590E0B9
:105800000E944C1720EA3DEF41E450E060E570E073
:1058100080E590E00E944C1720E030E04FE350E03C
:1058200060E570E080E590E00E944C1720EE3FEFCD
:1058300046E050E060E570E080E590E00E944C17A3
:10584000E12CF12C00E510E020EA30E040E550E0EA
:1058500060E070E081E594E00E94CF1090EEE92EC8
:10586000FF24FA9400E110E025E330E04EE450E03C
:1058700066E370E081E594E00E94CF108AE090E05A
:1058800090935E0480935D0427E330E030936004DE
:1058900020935F0463E272E081E594E00E94C2110C
:1058A00086E190E090935E0480935D0480E290E056
:1058B0009093600480935F0466E372E081E594E076
:1058C0000E94C2118AE290E090935E0480935D048E
:1058D0000FE010E01093600400935F0465E272E053
:1058E00081E594E00E94C21181E490E090935E040F
:1058F00080935D0427E0A22EB12CB0926004A092A8
:105900005F0467E272E081E594E00E94C2118AE5DB
:1059100090E090935E0480935D04B0926004A09246
:105920005F0463E972E081E594E00E94C21181E7BF
:1059300090E090935E0480935D0410936004009364
:105940005F0469E272E081E594E00E94C21184E89C
:1059500090E090935E0480935D04D0926004C092C6
:105960005F046BE272E081E594E00E94C21101E104
:1059700010E020E230E04BE650E060E470E081E5CA
:1059800094E00E94260603E010E024E030E048E6C0
:1059900050E064E470E081E594E00E94260624E093
:1059A00030E048E650E068E570E081E594E00E9470
:1059B0002606C12CD12C31E8E32EF12C0FE910E0A2
:1059C0002CE130E04FE950E06BE270E082E890E0DB
:1059D0000E943D152FE130E04CE050E065E470E0BE
:1059E00088E890E00E944C174FE1C42ED12C5FE371
:1059F000E52EF12C01E910E02DE230E048E850E01E
:105A00006FE370E08FE790E00E943D154DE950E0B4
:105A100068E870E083E790E00E941417C12CD12C55
:105A200065E6E62EF12C0BE910E028E730E048E8C7
:105A300050E065E670E084E790E00E943D1541E2A9
:105A400050E06EE770E088E890E00E947E19E12C5B
:105A5000F12C06E210E02FE030E041E650E064E691
:105A600070E081E594E00E94CF1008E010E02AE0A9
:105A700030E041E650E06EE970E081E594E00E949C
:105A8000CF108DE890E090935E0480935D0478E7FA
:105A9000A72EB12CB0926004A0925F048FEF97E024
:105AA00090936404809363049093620480936104F0
:105AB0006AE072E081E594E00E94C2114BE250E09E
:105AC00066E170E081E090E00E941417E5E6EE2EBA
:105AD000F12C0AE210E028E730E046E150E065E60C
:105AE00070E082E090E00E943D1541E250E06EE7F8
:105AF00070E086E190E00E947E19E12CF12C06E234
:105B000010E02FE030E043E650E06CE270E081E529
:105B100094E00E94CF1003E010E021E030E043E683
:105B200050E060E070E081E594E00E94CF1020EE4C
:105B30003FEF4FE550E06BE170E081E594E00E94BB
:105B4000660A20EE3FEF4FE550E061E170E081E54D
:105B500094E00E94660A20EE3FEF41E650E06AE0E2
:105B600070E081E594E00E94660A20EE3FEF41E696
:105B700050E062E270E081E594E00E94660A1092D3
:105B80005E0410925D04B0926004A0925F0462E033
:105B900072E081E594E00E94C21110921B01109204
:105BA0005903109258031092570310925603109203
:105BB0005403109253031092520310925103109207
:105BC0004F0310924E0310924B0310924A0310920F
:105BD00044031092450310924603109247038091AC
:105BE0003F03909140030B9709F061C0109240036E
:105BF00010923F0368E372E08EEA93E00E94C211C4
:105C00000E94C50A80914C0390914D038B30910501
:105C10002CF010924D0310924C0349C001969093C2
:105C20004D0380934C0343C067E872E08EEA93E033
:105C30000E94C2110E94DC0A11E01093650420E06A
:105C400038EF30936404209363043093620420930C
:105C5000610484E190E090935E0480935D042EE102
:105C600030E03093600420935F0466E472E081E5E5
:105C700094E00E94AE1184E190E090935E048093E2
:105C80005D042CE330E03093600420935F0467E50B
:105C900072E081E594E00E94AE1164EF71E080E073
:105CA00090E00E94B1120E94C50A10931B010E944D
:105CB0005F0F0C941F1B88E591E090938104809303
:105CC000800480E894E00C94AF134F925F926F923F
:105CD0007F928F929F92AF92BF92CF92DF92EF927C
:105CE000FF926B017C019B01AC010E9478338823F9
:105CF00019F062E373E01AC046015701E894B7F85F
:105D00002FEF3FEF4FE75FE7C501B4010E94783303
:105D1000811112C02FEF3FEF4FE75FE7C501B401DC
:105D20000E945B31181644F466E373E081E594E069
:105D30000E9450117C018AC02FEF3FEF4FE75FE4D4
:105D4000C701B6010E94FE3218161CF46AE373E024
:105D5000EDCF2FEF3FEF4FE75FECC701B6010E9499
:105D60005B3187FDF3CF20E030E0A901C701B60128
:105D70000E945B3187FF0BC06DE281E594E00E94D9
:105D800049115C01F7FAF094F7F8F09402C0A12CE5
:105D9000B12C2AE037ED43EA5BE3C701B6010E946C
:105DA000EF302B013C010E94DE316B017C010E942F
:105DB0000D329B01AC01C301B2010E94EE302B01F8
:105DC0003C012AE0B701A60181E594E00E9465113B
:105DD0007C01EA0CFB1C6EE281E594E00E94491113
:105DE000E80EF91E20E030E040E251E4C301B201C8
:105DF0000E9403332B013C010E94DE314B01A12C98
:105E0000B12C2AE0B501A40181E594E00E9465115E
:105E1000E80EF91EC501B4010E940D329B01AC01D0
:105E2000C301B2010E94EE3020E030E040E251E4D4
:105E30000E9403330E94DE31AB0160E070E02AE093
:105E400081E594E00E946511E80EF91E6FEB71E0A8
:105E500081E594E00E9450118E0D9F1DFF90EF9000
:105E6000DF90CF90BF90AF909F908F907F906F907A
:105E70005F904F900895AF92BF92CF92DF92EF92D2
:105E8000FF920F931F93CF93DF935C016C0182E02D
:105E9000C80ED11C7B0101E110E020E030E04CE0B5
:105EA00050E0B60181E594E00E94F4070CE010E0B8
:105EB00021E042E050E06EE070E0C50101960E94F2
:105EC000C51322E042E050E06EE070E0C6010E949F
:105ED000C513DF91CF911F910F91FF90EF90DF904D
:105EE000CF90BF90AF9008951092B1031092B0037D
:105EF00088EE93E0A0E0B0E08093B2039093B30308
:105F0000A093B403B093B50320E231E03093AF0324
:105F10002093AE0325EC30E03093BB032093BA030B
:105F200024EC30E03093BD032093BC0320EC30E040
:105F30003093BF032093BE0321EC30E03093C103C4
:105F40002093C00322EC30E03093C3032093C203BC
:105F500026EC30E03093C5032093C4031092C703AE
:105F60001092C8031092C9031092CA0320E520932F
:105F70004B0410924C04109283041092820480937C
:105F8000840490938504A0938604B093870488E5E5
:105F900091E0909381048093800410929704109272
:105FA0009604109299041092980410929B041092F7
:105FB0009A0410929D0410929C0460919E046E7F3E
:105FC0006D7F60939E046695617081E0682783E031
:105FD0000E94451261E083E00E947512E2E4F6E05F
:105FE000E491E0939004EEE2F6E0E491F0E0EE0F4D
:105FF000FF1FE95EF94F85919491909392048093ED
:10600000910460E082E00E94751280919E0481FDFF
:1060100004C061E082E00E94451282E080938C041B
:10602000E1E4F6E0E491E0938D04EDE2F6E0E49142
:10603000F0E0EE0FFF1FEF5DF94F85919491909383
:106040008F0480938E04109254041092530420E81D
:1060500030E0309356042093550480EA90E090930A
:1060600058048093570430935A0420935904909312
:106070005C0480935B041092660410925E0410929C
:106080005D041092600410925F0481E080936504C7
:106090002FEF3FEF30936404209363043093620446
:1060A00020936104809367041092680410926A043C
:1060B0001092690420E331E030935204209351049C
:1060C0009AE09093750498E09093760499E0909309
:1060D000770480936C04109279041092780480E025
:1060E00090E00E9488308093500481E090E00E940C
:1060F000883080934F0482E090E00E948830809343
:106100004E0483E090E00E94883080934D0408950F
:10611000F999FECF92BD81BDF89A992780B508956F
:10612000262FF999FECF1FBA92BD81BD20BD0FB6B3
:10613000F894FA9AF99A0FBE01960895052E97FBE6
:106140001EF400940E94B53057FD07D00E94BD3068
:1061500007FC03D04EF40C94B53050954095309523
:1061600021953F4F4F4F5F4F0895909580957095C3
:1061700061957F4F8F4F9F4F0895A1E21A2EAA1B62
:10618000BB1BFD010DC0AA1FBB1FEE1FFF1FA217E7
:10619000B307E407F50720F0A21BB30BE40BF50BE4
:1061A000661F771F881F991F1A9469F7609570956D
:1061B000809590959B01AC01BD01CF010895A29FF0
:1061C000B001B39FC001A39F700D811D1124911DCB
:1061D000B29F700D811D1124911D08955058BB2749
:1061E000AA270E9406310C94B0320E94773238F010
:1061F0000E947E3220F039F49F3F19F426F40C946B
:1062000074320EF4E095E7FB0C946E32E92F0E9495
:10621000D53258F3BA17620773078407950720F041
:1062200079F4A6F50C94F7320EF4E0950B2EBA2F04
:10623000A02D0B01B90190010C01CA01A00111248C
:10624000FF27591B99F0593F50F4503E68F11A1638
:10625000F040A22F232F342F4427585FF3CF4695C9
:1062600037952795A795F0405395C9F77EF41F16EB
:10627000BA0B620B730B840BBAF09150A1F0FF0FB5
:10628000BB1F661F771F881FC2F70EC0BA0F621FA1
:10629000731F841F48F4879577956795B795F79591
:1062A0009E3F08F0B0CF9395880F08F09927EE0F26
:1062B0009795879508950E944A3208F481E00895E1
:1062C0000E948732E3950C94C1320E9479310C947C
:1062D000B0320E947E3258F00E94773240F029F4AA
:1062E0005F3F29F00C946E3251110C94F8320C94EB
:1062F00074320E94D53268F39923B1F3552391F398
:10630000951B550BBB27AA2762177307840738F024
:106310009F5F5F4F220F331F441FAA1FA9F335D081
:106320000E2E3AF0E0E832D091505040E695001C35
:10633000CAF72BD0FE2F29D0660F771F881FBB1FEF
:10634000261737074807AB07B0E809F0BB0B802DCD
:10635000BF01FF2793585F4F3AF09E3F510578F0F9
:106360000C946E320C94F8325F3FE4F3983ED4F311
:10637000869577956795B795F7959F5FC9F7880FCD
:10638000911D9695879597F90895E1E0660F771F1F
:10639000881FBB1F621773078407BA0720F0621BB0
:1063A000730B840BBA0BEE1F88F7E09508950E94DB
:1063B000DE316894B1110C94F83208950E94DD32F8
:1063C00088F09F5798F0B92F9927B751B0F0E1F0B6
:1063D000660F771F881F991F1AF0BA95C9F714C066
:1063E000B13091F00E94F732B1E008950C94F73289
:1063F000672F782F8827B85F39F0B93FCCF386959F
:1064000077956795B395D9F73EF4909580957095FB
:1064100061957F4F8F4F9F4F0895E89409C097FB78
:106420003EF490958095709561957F4F8F4F9F4F6B
:106430009923A9F0F92F96E9BB279395F6958795AF
:1064400077956795B795F111F8CFFAF4BB0F11F472
:1064500060FF1BC06F5F7F4F8F4F9F4F16C0882319
:1064600011F096E911C0772321F09EE8872F762F4F
:1064700005C0662371F096E8862F70E060E02AF090
:106480009A95660F771F881FDAF7880F969587957C
:1064900097F90895990F0008550FAA0BE0E8FEEF51
:1064A00016161706E807F907C0F012161306E407D8
:1064B000F50798F0621B730B840B950B39F40A26D1
:1064C00061F0232B242B252B21F408950A2609F4AF
:1064D000A140A6958FEF811D811D089597F99F67B3
:1064E00080E870E060E008959FEF80EC089500245C
:1064F0000A941616170618060906089500240A9429
:10650000121613061406050608950C9474320E94A0
:10651000DD32D8F3E894E0E0BB279F57F0F02AED96
:106520003FE049EC06C0EE0FBB0F661F771F881FC8
:1065300028F0B23A62077307840728F0B25A620B58
:10654000730B840BE3959A9572F7803830F49A9523
:10655000BB0F661F771F881FD2F790480C947F33BC
:10656000092E0394000C11F4882352F0BB0F40F461
:10657000BF2B11F460FF04C06F5F7F4F8F4F9F4FA1
:106580000895EF93E0FF07C0A2EA2AED3FE049EC4F
:106590005FEB0E9406310E94B0320F90039401FC21
:1065A0009058E8E6F0E00C948B3357FD9058440F78
:1065B000551F59F05F3F71F04795880F97FB991F62
:1065C00061F09F3F79F0879508951216130614061F
:1065D000551FF2CF4695F1DF08C0161617061806AC
:1065E000991FF1CF86957105610508940895E89487
:1065F000BB2766277727CB0197F908950E944A3277
:1066000008F48FEF08950E9416330C94B0320E9464
:10661000773238F00E947E3220F0952311F00C94EE
:106620006E320C94743211240C94F8320E94D532DC
:1066300070F3959FC1F3950F50E0551F629FF001D5
:10664000729FBB27F00DB11D639FAA27F00DB11DEE
:10665000AA1F649F6627B00DA11D661F829F222777
:10666000B00DA11D621F739FB00DA11D621F839FFE
:10667000A00D611D221F749F3327A00D611D231FD4
:10668000849F600D211D822F762F6A2F11249F5722
:1066900050409AF0F1F088234AF0EE0FFF1FBB1F25
:1066A000661F771F881F91505040A9F79E3F5105E4
:1066B00080F00C946E320C94F8325F3FE4F3983E15
:1066C000D4F3869577956795B795F795E7959F5F8E
:1066D000C1F7FE2B880F911D9695879597F9089520
:1066E0009F930E9487320F9007FCEE5F0C94C1329B
:1066F0000E944A32880B990B08959F3F31F09150C8
:1067000020F4879577956795B795880F911D969595
:10671000879597F908959F938F937F936F93FF9336
:10672000EF939B01AC010E940333EF91FF910E9414
:106730009F332F913F914F915F910C940333DF93DF
:10674000CF931F930F93FF92EF92DF927B018C0107
:10675000689406C0DA2EEF010E941633FE01E89419
:10676000A5912591359145915591A6F3EF010E9490
:106770000631FE019701A801DA9469F7DF90EF90E6
:10678000FF900F911F91CF91DF91089597FB072EF6
:1067900016F4009407D077FD09D00E94E13307FC7E
:1067A00005D03EF4909581959F4F08957095619521
:1067B0007F4F08950E94DF30B7FF0895821B930B2F
:1067C0000895AA1BBB1B51E107C0AA1FBB1FA61738
:1067D000B70710F0A61BB70B881F991F5A95A9F78A
:1067E00080959095BC01CD010895EE0FFF1F059097
:1067F000F491E02D099481E090E0F8940C94003439
:1068000013E0CBE2D3E004C0FE010E94F5332196F1
:0A681000CC32D107C9F7F894FFCF8E
:10681A000000803F01001401000100010001000195
:10682A0000010001005000500001000100000000BA
:10683A00F60E720EBF0E9D0EB10E3D0F0000000047
:10684A004F05720E660A23081C08F407100804088C
:10685A002408F30784107D10120ABE09CF105D10B8
:10686A008506260600000000D00F720E24103C1088
:10687A00B70FCF0F536F66747761726520536572D5
:10688A0069616C20506F7274204F70656E65640088
:10689A00536176696E672073657474696E67732EC7
:1068AA002E2E2000536176696E67207365747469B1
:1068BA006E677300202D20446F6E65210064617934
:1068CA006C75782073657474696E67733A20000D6D
:1068DA000A006E696768746C7578207365747469E8
:1068EA006E67733A20003A20200900536372656587
:1068FA006E20300054505300303020202500424191
:10690A0054002020202020560052504D00202030D4
:10691A003000564143003020200041465200576162
:10692A007465720041697200504F54005363726576
:10693A00656E2031003300340036003700380053CA
:10694A00637265656E203200200950617373204DB1
:10695A006164653A20004E6F20636F6E6E656374E2
:10696A00696F6E20746F0053706974726F6E696319
:10697A007320556E69740053656E64696E672032C0
:10698A0035320053706974726F6E69637300424FD7
:10699A004F54494E472E2E2E0053656E64696E671A
:1069AA002032353500547970653A2020004E6F49FF
:1069BA006E697400454355005443550043414D00E8
:1069CA0054487857004D6F64656C3A2000454D5520
:1069DA0000546974616E0056656E7573004D657278
:1069EA006375727900506C75746F004D65726375CA
:1069FA00727932004E657074756E65004E657074FA
:106A0A00756E6532004669726D77617265205665EA
:106A1A007273696F6E3A2000446973706C617920F1
:106A2A00556E69742076312E31006461796C7578FF
:106A3A003A00206E696768746C75783A00202800FD
:0E6A4A0029006E616E00696E66006F76660050
:00000001FF
